:0400000057EF00F0C6
:10000800065A065A065A065A065A065A065AAF5148
:10001800065A065A065A065A065A065A065A065AD8
:10002800065A065A065A065A065A065A065A065AC8
:10003800065A065A065AED54065A065A065A0A57D6
:10004800065A065A9759065A2B00065A065A065A4D
:10005800065A065A065A065A065A065A065A065A98
:10006800065A065A065A065A065A065A065A065A88
:10007800065A065A2B00065A065A065A2B002B0017
:100088002B002B002B002B002B002B00065A065AA6
:100098003D59065A065A065A2B002B002B002B00F6
:0A00A800065A065AFF004DEFA5F0BE
:10F3F4000000000000001B1B0000181818181B1B3D
:10F404000000030303031B1B00001B1B1B1B1B1B14
:10F4140000040E1F0404040400040404041F0E0466
:10F42400001112140B110203000E0A0E000000005A
:10F43400005067018E6401B466010E450146520115
:10F44400DC57013C5301186701F86701F4670114A4
:10F454006501B86701C067010A6701B06701FA6610
:10F4640001805B01BA5901EA66010080C094D4208E
:10F474002000204861726477617265203A2042411D
:10F4840053452031384632374B34322C20493243ED
:10F49400313A20204C4344347832302C494E4132A6
:10F4A40032362C4942542032204D6F736665742CD9
:10F4B4004D43503233303137202B20554152543193
:10F4C4000D0A20536368656D613A20436172746567
:10F4D4005F506F727461696C5F325F56616E746104
:10F4E40075785F3234765F482D656E2D4D4F5346E7
:10F4F40045545F494E413232362D484950343038F4
:10F50400325F46515033304E30364C5F56352E30D4
:10F514002E332E70646620627920482E542E0D0AF4
:10F524000D0A0020417574726573203A0D0A20207B
:10F534004C43445F34626974735F4932435F3230D1
:10F5440032352D30352C2055415254315F46756E7D
:10F554006374696F6E732E68202C206D63632E684C
:10F564002C0D0A0045434F2E2E2E2E00424152529E
:10F57400455F470042415252455F44004241525266
:10F5840045474400464C454348204800464C4543C3
:10F59400485F4200312F3248657572004445475236
:10F5A40045432000204C43445F63686172735F539A
:10F5B400706563696175785F323032342E682C204F
:10F5C4002020456570726F6D203A20456570726F1A
:10F5D4006D2E2E2E2E2E2E2E2E2E2E2E2020200D53
:10F5E4000A00205241303D2E2E2E5241313D416EB3
:10F5F400616C6F67202C5241343D6C65642C524120
:10F60400332E2E2E5243363D5458205541525431F8
:10F61400205243373D525820554152540D0A002080
:10F624004120696E636C7572653A200D0A20446945
:10F63400616C6F6775655F4F706572617465757233
:10F644005F50435F7669615F554152545F32303297
:10F65400332D303930350D0A0D0A002044697265A6
:10F6640063746F7279203A433A5C4D504C4142586E
:10F674005F50726F6A656374735C31384632374B1E
:10F6840034325F504D575F434350313233345F322D
:10F694003032350D0A00204241534520313846327C
:10F6A400374B3432202B204C4344345832302B20F7
:10F6B40050574D312C322C332C3420416E616C6FF9
:10F6C40067205241302C312C322C330D0A00204C4F
:10F6D40043442034783230206275732049324331F8
:10F6E400204857203A205243333D53434C2C524335
:10F6F400343D5344410D0A002050726F6A656374AF
:10F70400203A2031384632374B34325F504D575F00
:10F71400434350313233345F323032350D0A0020E6
:10F72400536F75726365203A20206D61696E2E6394
:10F73400202C20726576203A5F3235303531320D17
:10F744000A0020436F6E6669672020496E746572F3
:10F754006E616C20466F73632036344D487A0D0A0F
:10F7640000202020202020202020202020202020B5
:10F774002020202020002052423020414C45525469
:10F7840020696E7075740D0A002052617070656C8A
:10F79400203A2063646520504D57793D5858585895
:10F7A400206176656320793D63686F697820504DE8
:10F7B400572031206F7520322065742020787878A6
:10F7C40078202076616C65757220647574792030B8
:10F7D400303030206120313031350D0A002054653D
:10F7E400737420646966666572656E7465732076E9
:10F7F400616C6575727320646520447574792D633A
:10F8040079636C6520766961206C6520636C617630
:10F81400696572207465726D696E616C205941541A
:10F82400200D0A0020456E7472657220756E652085
:10F8340076616C6575722050574D793D787878788B
:10F844002070756973203C656E7465723E20617624
:10F85400656320793D31206F752032206175206306
:10F864006C61766965720D0A0020496E69742049DD
:10F874004E41323236206D657375726520646520A1
:10F88400636F7572616E7420766961204932432C0E
:10F89400207368756E74206465203135306D562090
:10F8A400706F75203135416D70730D0A002043610E
:10F8B4006C6962726174696F6E20726567697374D2
:10F8C4006572203035682028706F757220736875F2
:10F8D4006E7420302C3031206F686D2020657420C8
:10F8E4003820416D707329200D0A002050574D3285
:10F8F4003D58585858202020617665632058585840
:10F904002064652030303030206131303030207058
:10F914006F75722052433120646520302520613197
:10F92400303025200D0A002050574D313D5858588D
:10F93400582020206176656320585858206465203B
:10F944003030303020613130303020706F757220AB
:10F954005243322064652030252061313030252027
:10F964000D0A002041637469766572206C6120730E
:10F974006F727469652050574D79206176656320F4
:10F984004D413D312020202028617272657420761B
:10F994006961204D413D30290D0A0020416C65729A
:10F9A40074204D41534B5F454E5F5245472072656D
:10F9B40067697374657220303768203C2D203234B7
:10F9C400303020706F757220302E3620410D0A00C1
:10F9D4002076657273696F6E2050726F746F7479DC
:10F9E4007065203A204C434420426C6575206120A8
:10F9F4006C27616472657373652030783237202117
:10FA04000D0A0020496E697469616C6973617469D7
:10FA14006F6E2050574D312C32206176656320463D
:10FA240052657120332C394B487A202854696D650E
:10FA34007232290D0A00204D61736B2F416C65727F
:10FA44007420204D41534B5F454E5F524547207211
:10FA54006567697374657220303668203C2D2030E8
:10FA640078383030310D0A00204572726575722085
:10FA7400646520536169736965202063686F6978E0
:10FA8400204343502025632076616C6575722050B5
:10FA9400574D202535640D0A0020436F6E66696753
:10FAA4002020494E413232365F434F4E465F524525
:10FAB400472C3078343346462028776173203078D9
:10FAC4003431323720290D0A00200D0A536571752F
:10FAD400656E6365206427496E6974204C43442035
:10FAE40034783230207669612049324331205043E2
:10FAF40046383537340D0A00204020646563696D4B
:10FB0400616C20232534752020736F697420404470
:10FB14006576696365203762697473203D203058C7
:10FB240025303258200020256C752E256C75206DEB
:10FB340053202020434150423D2030782530325814
:10FB440020202049545F466C6167203D2030782591
:10FB540030325800204368617267656D656E7420A9
:10FB64006361726163746572657320537065636960
:10FB74006175782020656E20434752414D0D0A007F
:10FB840020436F6D70696C65642025732061742057
:10FB9400257320555443202076657273696F6E2057
:10FBA400584338203A2564200D0A00204D413D3148
:10FBB400206F752030202020313D4D6172636865CF
:10FBC400206F7520303D41727265742050574D206E
:10FBD4000D0A000D0A2054657374206368726F6EF9
:10FBE4006F206176656320544D5236207820313081
:10FBF40020626F75636C65730D0A0020546573741D
:10FC04002070726573656E636520646576696365EB
:10FC140073207375722042757320493243310D0A83
:10FC2400002046696E20646520706172616D6574A0
:10FC34007261676520494E413232362E2E2E204F96
:10FC44004B0D0A0D0A000D0A2046696E2074656D7D
:10FC5400706F2064652031207365632076696120AC
:10FC6400544D5236200D0A00206164726573736529
:10FC7400204C43443D20256420736F697420305820
:10FC840025303258200D0A0020536575696C2064B4
:10FC940027616C657274652025332E336620416DAF
:10FCA40070657265730D0A00204D65737572652069
:10FCB400646520636F7572616E742025203564203D
:10FCC4006D41200D0A00202A2050574D32207375B3
:10FCD40072205243312028544D5232293D30252080
:10FCE4000D0A00202A2050574D312073757220527E
:10FCF40043322028544D5232293D3025200D0A002C
:10FD0400456570726F6D2032344C437878782032B8
:10FD140035366B206F75203531324B0020494E410A
:10FD2400204D616E7566616374756572202030784C
:10FD3400253034580D0A0020494E41204964656E2F
:10FD440074696669616E74203078253034580D0A00
:10FD54000020496E697420534D543120636F6D70D7
:10FD640074657572203234620D0A0020504346389F
:10FD740037353420666F72204C4344203278313654
:10FD840063617273000D0A2052415A20616C6172E2
:10FD94006D65202C526573746172740D0A00204DD8
:10FDA40043503233303137203220706F72747320F5
:10FDB40038626974730020496E69745F493243285C
:10FDC40029203130304B687A3B0D0A0050574D32B0
:10FDD4002D52433120202534642025332E316625CD
:10FDE400630050574D312D52433220202534642076
:10FDF40025332E3166256300494E41323236204385
:10FE0400757272656E742073656E736F72004361F0
:10FE1400726163746572657320537065636961759B
:10FE24007820002025322E32662056202025322EBE
:10FE34003366204120202E00504D57322D5243313D
:10FE4400202534642025332E316625630050574D18
:10FE5400312D524332202534642025332E3166253A
:10FE64006300205072657320456E746572206B6563
:10FE74007920210D0A0020534D5431204E62205424
:10FE840069637320256C750D0A0056657273696F7A
:10FE94006E2050726F746F74797065202100204950
:10FEA4006E69742054524D36203130306D530D0A32
:10FEB4000050434638353734412038626974732022
:10FEC400492F4F0020495442322044697361626CC7
:10FED4006564200D0A002050726573656E74617448
:10FEE400696F6E203A0D0A004C4344203231313997
:10FEF40020327831366361727300204954423220D3
:10FF0400456E61626C6564200D0A0020496E697457
:10FF1400204D435032333031370D0A0050434638B8
:10FF240035373420386269747320494F004E3D25BB
:10FF34003564202050574D313D202534640045451B
:10FF440050524F4D2035313262797465730020531D
:10FF54006575696C3D25332E336620002045727229
:10FF64006575722063780D0A004F4C454420535345
:10FF740044313330360020536169736965204F4B37
:10FF840020006E6F6E20636F6E6E752021004D61D0
:10FF9400792031322032303235002050574D323DF5
:10FFA40020252034640052544320445333323331E7
:10FFB4000031373A33373A353900414C4552540D04
:10FFC4000A0048656C700D0A0052656375203A009A
:10FFD400494E46004E414E00696E66006E616E00E9
:10FFE4006C6C7300202E31006C58006C64006C66DD
:0BFFF400006C69006C75006C78000068
:020000040001F9
:10000000C551D96EDA6A6F007BFFF6FF6F0077FF8C
:10001000F7FF000EF86E0800F550250AD8A4BEEFD1
:1000200085F0C551D96EDA6ADE2A000EDD22000E97
:10003000416E000E406E40C044F041C045F0426841
:100040004368000ED96F000E13D04480C551D96E9D
:10005000DA6ADE2A000EDD2231D04482F7D74484EA
:10006000F5D74486F3D74488F1D7000ED96F010E37
:10007000D86F24D0C551D96EDA6A6F007BFFF6FFC6
:100080006F0077FFF7FF000EF86E0800F550C86F9D
:10009000C96BC951000AD8A4E8D7C851200AD8B4FE
:1000A000E0D7030AD8B4DFD7080AD8B4D8D7060AED
:1000B000D8B4CBD71D0AD8B4D0D7D7D7D851D911F7
:1000C000D8B4D8D744B04492C551D96EDA6A6F001B
:1000D0007BFFF6FF6F0077FFF7FF000EF86E08005A
:1000E000F5502A0AD8A42AD0C551D96EDA6ADE2A78
:1000F000000EDD2260001BF3D9FF60001FF3DAFF62
:100100006F007CFFC8F0020EDE266F007CFFC9F096
:10011000000EDD22600023F3D9FF600027F3DAFF31
:100120006F0078FF40F06F0074FF41F041AE3AD0AD
:100130004480406C411ED8B0412A34D0C551D96E9C
:10014000DA6A6F0078FF18F06F0074FF19F00EEC98
:100150009FF018C040F019C041F006D0C551D96ECB
:10016000DA6ADE2A000EDD22D00E0001C86FFF0E13
:10017000C96FC551D96EDA6A6F007BFFF6FF6F0059
:1001800077FFF7FF000EF86E0800F550CA6FCB6BD3
:10019000C851CA27C951CB23CB5104E10A0ECA5D0D
:1001A000D8A0DCD7C551D96EDA6A6F007BFFF6FFA5
:1001B0006F0077FFF7FF000EF86E0800F5502E0A6B
:1001C000D8A471D0000E436E000E426EC551D96E98
:1001D000DA6ADE2A000EDD22C551D96EDA6A6F00B6
:1001E0007BFFF6FF6F0077FFF7FF000EF86E080049
:1001F000F5502A0AD8A423D0C551D96EDA6ADE2A6E
:10020000000EDD2260001BF3D9FF60001FF3DAFF50
:100210006F007CFFC8F0020EDE266F007CFFC9F085
:10022000000EDD22600023F3D9FF600027F3DAFF20
:100230006F0078FF42F06F0074FF43F034D0C55177
:10024000D96EDA6A6F0078FF18F06F0074FF19F04A
:100250000EEC9FF018C042F019C043F006D0C55113
:10026000D96EDA6ADE2A000EDD22D00E0001C86FD8
:10027000FF0EC96FC551D96EDA6A6F007BFFF6FFBA
:100280006F0077FFF7FF000EF86E0800F550CA6F99
:10029000CB6BC851CA27C951CB23CB5104E10A0EFD
:1002A000CA5DD8A0DCD7C551D96EDA6A6F007BFF72
:1002B000F6FF6F0077FFF7FF000EF86E0800F550AD
:1002C000176E186AB2ECAFF01750E86FE851D8B467
:1002D0003DD0C551D96EDA6A6F0078FFC8F06F0063
:1002E00074FFC9F0010EC827000EC923600023F374
:1002F000F6FF600027F3F7FF000EF86E0800F550D8
:10030000176E186AB2ECAFF01750E96FE951D8B424
:100310001DD0C551D96EDA6A6F0078FFC8F06F0042
:1003200074FFC9F0020EC827000EC923600023F332
:10033000F6FF600027F3F7FF000EF86E0800F55097
:10034000176E186AB2ECAFF01750EA6FC551D96E4C
:10035000DA6A6F007BFFF6FF6F0077FFF7FF000E92
:10036000F86E0800F550630AD8A42BD0C551D96E99
:10037000DA6ADE2A000EDD2260001BF3D9FF60007E
:100380001FF3DAFF6F007CFFC8F0020EDE266F005D
:100390007CFFC9F0000EDD22600023F3D9FF60006E
:1003A00027F3DAFFDF50F36FC3C01AF0C4C01BF0AD
:1003B000F3C01CF0F2ECA6F01AC0C3F01BC0C4F0EE
:1003C0001200C551D96EDA6A6F007BFFF6FF6F002D
:1003D00077FFF7FF000EF86E0800F550640AD8B4F6
:1003E00010D0C551D96EDA6A6F007BFFF6FF6F003F
:1003F00077FFF7FF000EF86E0800F550690AD8A4E1
:1004000046D0C551D96EDA6ADE2A000EDD226000C0
:100410001BF3D9FF60001FF3DAFF6F007CFFC8F009
:10042000020EDE266F007CFFC9F0000EDD226000A8
:1004300023F3D9FF600027F3DAFF6F0078FFDCF0C9
:100440006F0074FFDDF0000EDDBFFF0EDE6FDF6FAB
:10045000E06FE16FE26FE36FC3C02CF0C4C02DF01A
:10046000DCC02EF0DDC02FF0DEC030F0DFC031F098
:10047000E0C032F0E1C033F0E2C034F0E3C035F068
:1004800024EC99F02CC0C3F02DC0C4F01200C5516B
:10049000D96EDA6A6F0078FF11F06F0074FF12F006
:1004A000EF0E136EFF0E146E000E166E020E156E1A
:1004B0007BECA1F011501210D8B418D00001C55136
:1004C000D96EDA6A6F0078FF11F06F0074FF12F0D6
:1004D000F50E136EFF0E146E000E166E020E156EE4
:1004E0007BECA1F011501210D8A44CD00001C551E2
:1004F000D96EDA6A020EDE26000EDD2260001BF3E2
:10050000D9FF60001FF3DAFF6F007CFFC8F0040E14
:10051000DE266F007CFFC9F0000EDD22600023F3B1
:10052000D9FF600027F3DAFF6F0078FFCAF06F0091
:1005300078FFCBF06F0078FFCCF06F0078FFCDF044
:10054000CAC0CEF0CBC0CFF0CCC0D0F0CDC0D1F07F
:10055000D26BD1BFD269D2C0D3F0D2C0D4F0D2C056
:10056000D5F0CEC0DCF0CFC0DDF0D0C0DEF0D1C021
:10057000DFF0D2C0E0F0D3C0E1F0D4C0E2F0D5C0EB
:10058000E3F06AD7660E0001E819D8A44CD0C55133
:10059000D96EDA6A6F007BFFF6FF6F0077FFF7FF17
:1005A000000EF86E08006F00D4FFF3F0C551D96E4D
:1005B000DA6ADE2A000EDD2260001BF3D9FF60003C
:1005C0001FF3DAFF6F007CFFC8F0040EDE266F0019
:1005D0007CFFC9F0000EDD22600023F3D9FF60002C
:1005E00027F3DAFF6F0078FFE4F06F0078FFE5F0A3
:1005F0006F0078FFE6F06F0078FFE7F0C3C085F08A
:10060000C4C086F0E4C087F0E5C088F0E6C089F099
:10061000E7C08AF0F3C08BF0DBEC85F085C0C3F057
:1006200086C0C4F01200E80E116E126AF20E136E4C
:10063000FF0E146E000E166E020E156E7BECA1F00E
:1006400011501210D8A45FD00001C551D96EDA6ADA
:100650006F0078FFC8F06F0074FFC9F0010EC82763
:10066000000EC923600023F3F6FF600027F3F7FFB5
:10067000000EF86E08006F00D4FFF3F0BF0EC86FD5
:10068000FF0EC96FC551D96EDA6A6F007BFFF6FFA6
:100690006F0077FFF7FF000EF86E0800F550CA6F85
:1006A000CB6BC851CA27C951CB23CB5102E11A0EDB
:1006B000CA5D60001BF3D9FF60001FF3DAFF6F0013
:1006C0007CFFC8F0040EDE266F007CFFC9F0000E30
:1006D000DD22600023F3D9FF600027F3DAFF6F000B
:1006E00078FFE4F06F0078FFE5F06F0078FFE6F048
:1006F0006F0078FFE7F0C551D96EDA6A020EDE2688
:10070000000EDD227BD70001C551D96EDA6A6F0079
:100710007BFFF6FF6F0077FFF7FF000EF86E080013
:10072000F550730AD8B417D0C551D96EDA6A6F0084
:1007300078FF11F06F0074FF12F0E40E136EFF0EDD
:10074000146E000E166E030E156E7BECA1F01150A8
:100750001210D8A44BD00001C551D96EDA6A6F00CF
:100760007BFFF6FF6F0077FFF7FF000EF86E0800C3
:10077000F550730AD8B404D0000EDB6F030E03D01B
:10078000000EDB6F010EDA6FC551D96EDA6ADA51ED
:10079000DE26DB51DD2260001BF3D9FF60001FF372
:1007A000DAFF6F007CFFC8F0020EDE266F007CFFD0
:1007B000C9F0000EDD22600023F3D9FF600027F3AB
:1007C000DAFF6F0078FFD6F06F0074FFD7F0C3C078
:1007D0001AF0C4C01BF0D6C01CF0D7C01DF0C6EC88
:1007E0009DF01AC0C3F01BC0C4F012000001C55137
:1007F000D96EDA6A6F007BFFF6FF6F0077FFF7FFB5
:10080000000EF86E0800F550750AD8A447D0C551FF
:10081000D96EDA6ADE2A000EDD2260001BF3D9FFF2
:1008200060001FF3DAFF6F007CFFC8F0020EDE26C7
:100830006F007CFFC9F0000EDD22600023F3D9FFBA
:10084000600027F3DAFF6F0078FFCAF06F0074FFD3
:10085000CBF0CAC0EBF0CBC0ECF0ED6BEE6BEF6B06
:10086000F06BF16BF26BC3C02CF0C4C02DF0EBC089
:100870002EF0ECC02FF0EDC030F0EEC031F0EFC044
:1008800032F0F0C033F0F1C034F0F2C035F04EEC8D
:100890009BF02CC0C3F02DC0C4F01200C551D96E1E
:1008A000DA6A6F0078FF11F06F0074FF12F0F80E33
:1008B000136EFF0E146E000E166E020E156E7BEC9C
:1008C000A1F011501210D8A433D00001C551D96E37
:1008D000DA6A020EDE26000EDD2260001BF3D9FF6D
:1008E00060001FF3DAFF6F007CFFC8F0040EDE2605
:1008F0006F007CFFC9F0000EDD22600023F3D9FFFA
:10090000600027F3DAFF6F0078FFCAF06F0078FF0E
:10091000CBF06F0078FFCCF06F0078FFCDF0CA51BC
:10092000EB6FCB51EC6FCC51ED6FCD51EE6F97D794
:100930000001C551D96EDA6A6F007BFFF6FF6F00C8
:1009400077FFF7FF000EF86E0800F550780AD8B46C
:1009500010D0C551D96EDA6A6F007BFFF6FF6F00C9
:1009600077FFF7FF000EF86E0800F550580AD8A47C
:1009700058D0C551D96EDA6A6F007BFFF6FF6F0061
:1009800077FFF7FF000EF86E08006F00D4FFF3F05A
:10099000C551D96EDA6ADE2A000EDD2260001BF333
:1009A000D9FF60001FF3DAFF6F007CFFC8F0020E72
:1009B000DE266F007CFFC9F0000EDD22600023F30D
:1009C000D9FF600027F3DAFF6F0078FFCAF06F00ED
:1009D00074FFCBF0CAC0EBF0CBC0ECF0ED6BEE6B6C
:1009E000EF6BF06BF16BF26BC3C02CF0C4C02DF059
:1009F000EBC02EF0ECC02FF0EDC030F0EEC031F0C7
:100A0000EFC032F0F0C033F0F1C034F0F2C035F096
:100A1000F3C036F047EC9AF02CC0C3F02DC0C4F000
:100A20001200C551D96EDA6A6F0078FF11F06F00BD
:100A300074FF12F0FB0E136EFF0E146E000E166E96
:100A4000020E156E7BECA1F011501210D8B418D024
:100A50000001C551D96EDA6A6F0078FF11F06F009E
:100A600074FF12F0EC0E136EFF0E146E000E166E75
:100A7000020E156E7BECA1F011501210D8A44CD0D0
:100A80000001C551D96EDA6A6F0078FFC8F06F00B7
:100A900074FFC9F0010EC827000EC923600023F3BC
:100AA000F6FF600027F3F7FF000EF86E08006F00F6
:100AB000D4FFF3F0C551D96EDA6A020EDE26000EBD
:100AC000DD2260001BF3D9FF60001FF3DAFF6F0027
:100AD0007CFFC8F0040EDE266F007CFFC9F0000E1C
:100AE000DD22600023F3D9FF600027F3DAFF6F00F7
:100AF00078FFCAF06F0078FFCBF06F0078FFCCF082
:100B00006F0078FFCDF0CA51EB6FCB51EC6FCC5139
:100B1000ED6FCD51EE6F64D70001C551D96EDA6A21
:100B20006F007BFFF6FF6F0077FFF7FF000EF86E98
:100B30000800F550250AD8A416D0C551D96EDA6A36
:100B4000DE2A000EDD22000E126E250E116EC3C0CD
:100B500013F0C4C014F0FEECA5F0000E0001C46F49
:100B6000010EC36F1200C551D96EDA6ADE2A000E7B
:100B7000DD22000EC46F000EC36F1200C551D96E86
:100B8000DA6A6F007BFFF6FF6F0077FFF7FF000E5A
:100B9000F86E0800F550116E126AC3C013F0C4C09D
:100BA00014F0FEECA5F00001C551D96EDA6ADE2A18
:100BB000000EDD22D2D7000EA66F000EA56F87C0F3
:100BC000B7F088C0B8F089C0B9F08AC0BAF0BAAF3F
:100BD00016D0000EA66F010EA56FB7C011F0B8C0F9
:100BE00012F0B9C013F0BAC014F098ECB1F011C013
:100BF000B7F012C0B8F013C0B9F014C0BAF0000ECC
:100C0000BE6F000EBD6F40C0A9F041C0AAF0A55153
:100C1000A611D8A402D044A413D0A551A611D8A4DB
:100C200004D0000E926F2B0E03D0000E926F2D0E8B
:100C3000916F91C080F2BD4BBE2BA907D8A0AA0727
:100C4000B7C011F0B8C012F0B9C013F0BAC014F0B8
:100C50002EECA4F011041210D8A443D0BF0E000152
:100C60008C6FFF0E8D6F8B518E6F8F6B8C518E271B
:100C70008D518F238F5111E11A0E8E5DD8B00DD09A
:100C8000800EBD25156E020EBE21166ED40E176E97
:100C9000FF0E186E1FECACF00CD0800EBD25156E4B
:100CA000020EBE21166EDC0E176EFF0E186E1FECC4
:100CB000ACF00001FD0EA927FF0EAA2385C021F08C
:100CC00086C022F0800E236E020E246EA9C025F08D
:100CD000AAC026F08CECA7F021C085F022C086F0D7
:100CE0001200B7C011F0B8C012F0B9C013F0BAC00A
:100CF00014F02EECA4F011501210D8A42CD0BF0E7A
:100D000000018C6FFF0E8D6F8B518E6F8F6B8C512E
:100D10008E278D518F238F5111E11A0E8E5DD8B021
:100D20000DD0800EBD25156E020EBE21166ED80E9A
:100D3000176EFF0E186E1FECACF0BBD7800EBD25F2
:100D4000156E020EBE21166EE00E176EFF0E186EA7
:100D50001FECACF0AED7000E0001BF6F000EC06FED
:100D6000800EC16F3F0EC26F000EBC6F000EBB6FD6
:100D7000B7C011F0B8C012F0B9C013F0BAC014F087
:100D8000000E156E000E166E000E176E000E186E19
:100D9000D7ECA7F0D8A01ED075D0BFC01FF0C0C040
:100DA00020F0C1C021F0C2C022F0000E236E000E60
:100DB000246E200E256E410E266E88EC93F01FC027
:100DC000BFF020C0C0F021C0C1F022C0C2F00001BD
:100DD000BB4BBC2BB7C038F0B8C039F0B9C03AF043
:100DE000BAC03BF0000E236E000E246E200E256E5E
:100DF000410E266EBFC01FF0C0C020F0C1C021F060
:100E0000C2C022F088EC93F01FC03CF020C03DF03F
:100E100021C03EF022C03FF0F5ECA2F0D8A01ED0D9
:100E2000BCD7BFC038F0C0C039F0C1C03AF0C2C0B2
:100E30003BF0000E3C6E000E3D6E200E3E6E410EED
:100E40003F6EB6EC96F038C0BFF039C0C0F03AC083
:100E5000C1F03BC0C2F0BB07D8A0BC07B7C038F098
:100E6000B8C039F0B9C03AF0BAC03BF0BFC03CF0EE
:100E7000C0C03DF0C1C03EF0C2C03FF0F5ECA2F0F2
:100E8000D8A0CFD78BC017F0186AB2ECAFF01750CC
:100E9000AC6FACC0ABF0670EAC19D8A419D04250FF
:100EA0004310D8A404D0000E436E010E426E43BE20
:100EB00005D0435008E14204D8B005D0000EA86F19
:100EC000060EA76F08D042C0A7F043C0A8F003D019
:100ED00043AEF9D7F3D7670EAC19D8A422D0BCAF74
:100EE00006D0FC0EBB5DFF0EBC59D8A018D0FF0E7B
:100EF0008C6FFF0E8D6FA7C08EF0A8C08FF08C5145
:100F00008E278D518F23BB518E5D8F51800A906F3C
:100F1000BC51800A9059D8A002D0660E01D0650E4F
:100F2000AB6FA7C09DF0A8C09EF0670EAC19D8A407
:100F300005D0660EAB19D8B4BCAF02D09D4B9E2B2A
:100F4000660EAB19D8A416D0BCAF0CD0000EBF6F84
:100F5000000EC06F800EC16F3F0EC26F000EBC6FDF
:100F6000000EBB6F670EAC19D8B404D0BB519D27DF
:100F7000BC519E23000EB66F000EB56FB7C0ADF02A
:100F8000B8C0AEF0B9C0AFF0BAC0B0F0BFC09FF00B
:100F9000C0C0A0F0C1C0A1F0C2C0A2F07AD0ADC064
:100FA00038F0AEC039F0AFC03AF0B0C03BF0BFC0CF
:100FB0003CF0C0C03DF0C1C03EF0C2C03FF0B6EC56
:100FC00096F038C071F039C072F03AC073F03BC08F
:100FD00074F026EC9CF071C0B1F072C0B2F073C036
:100FE000B3F074C0B4F0B1C011F0B2C012F0B3C02D
:100FF00013F0B4C014F094ECA4F011C0A3F012C02C
:10100000A4F0ADC038F0AEC039F0AFC03AF0B0C017
:101010003BF0BFC023F0C0C024F0C1C025F0C2C067
:1010200026F0B1C01FF0B2C020F0B3C021F0B4C0B0
:1010300022F088EC93F01FC03CF020C03DF021C0AE
:101040003EF022C03FF0F4ECAEF038C0ADF039C055
:10105000AEF03AC0AFF03BC0B0F0BFC038F0C0C097
:1010600039F0C1C03AF0C2C03BF0000E3C6E000E39
:101070003D6E200E3E6E410E3F6EB6EC96F038C0CF
:10108000BFF039C0C0F03AC0C1F03BC0C2F0B54BB0
:10109000B62B9D51B55DB651800A8C6F9E51800A6A
:1010A0008C59D8A07CD7BFC01FF0C0C020F0C1C0F1
:1010B00021F0C2C022F0000E236E000E246EA00E9E
:1010C000256E400E266E88EC93F01FC0B1F020C054
:1010D000B2F021C0B3F022C0B4F0ADC038F0AEC061
:1010E00039F0AFC03AF0B0C03BF0B1C03CF0B2C094
:1010F0003DF0B3C03EF0B4C03FF0F5ECA2F0D8A094
:1011000015D0ADC011F0AEC012F0AFC013F0B0C03A
:1011100014F0B1C015F0B2C016F0B3C017F0B4C0EF
:1011200018F0D7ECA7F0D8B0A3B108D0000EB16F7B
:10113000000EB26F000EB36F000EB46FB7C011F0A7
:10114000B8C012F0B9C013F0BAC014F0B1C015F0B5
:10115000B2C016F0B3C017F0B4C018F030EC95F080
:1011600011C0ADF012C0AEF013C0AFF014C0B0F0BB
:10117000ADC038F0AEC039F0AFC03AF0B0C03BF00F
:10118000000E236E000E246E200E256E410E266E7C
:101190009FC01FF0A0C020F0A1C021F0A2C022F08B
:1011A00088EC93F01FC03CF020C03DF021C03EF021
:1011B00022C03FF0F5ECA2F0D8A023D0BB4BBC2B53
:1011C0009FC01FF0A0C020F0A1C021F0A2C022F05B
:1011D000000E236E000E246E200E256E410E266E2C
:1011E00088EC93F01FC09FF020C0A0F021C0A1F0B8
:1011F00022C0A2F0660E0001AB19D8A402D09D4B0C
:101200009E2B9FC0BFF0A0C0C0F0A1C0C1F0A2C083
:10121000C2F0650EAB19D8B405D0BBC09BF0BCC002
:101220009CF004D0000E9C6F000E9B6F000E9A6F16
:10123000000E996F000E986F000E976F000EB66F3C
:10124000000EB56FC4D0ADC038F0AEC039F0AFC03D
:101250003AF0B0C03BF0BFC03CF0C0C03DF0C1C0F0
:101260003EF0C2C03FF0B6EC96F038C071F039C025
:1012700072F03AC073F03BC074F026EC9CF071C081
:10128000B1F072C0B2F073C0B3F074C0B4F0B1C0CA
:1012900011F0B2C012F0B3C013F0B4C014F094EC6B
:1012A000A4F011C0A3F012C0A4F044B80CD0A35114
:1012B000A411D8A408D0670EAC19D8B49CAF03D041
:1012C000974B982B39D099519A11D8B49CAF22D012
:1012D000800EBD25D96E020EBE21DA6E2E0EDF6E97
:1012E000BD4BBE2BA907D8A0AA07000E9A6F010E0E
:1012F000996F10D0800EBD25D96E020EBE21DA6E18
:10130000300EDF6EBD4BBE2BA907D8A0AA079707EA
:10131000D8A0980797519811D8A4ECD7800EBD2576
:10132000D96E020EBE21DA6EA351300FDF6EBD4BB7
:10133000BE2BA907D8A0AA07ADC038F0AEC039F0BF
:10134000AFC03AF0B0C03BF0BFC023F0C0C024F043
:10135000C1C025F0C2C026F0B1C01FF0B2C020F05D
:10136000B3C021F0B4C022F088EC93F01FC03CF071
:1013700020C03DF021C03EF022C03FF0F4ECAEF0C2
:1013800038C0ADF039C0AEF03AC0AFF03BC0B0F0FD
:10139000BFC038F0C0C039F0C1C03AF0C2C03BF0A5
:1013A000000E3C6E000E3D6E200E3E6E410E3F6EF6
:1013B000B6EC96F038C0BFF039C0C0F03AC0C1F00A
:1013C0003BC0C2F09B07D8A09C07B54BB62B9D51E4
:1013D000B55DB651800A8C6F9E51800A8C59D8B089
:1013E00008D0BEBF30D7BE5104E14B0EBD5DD8A0C2
:1013F0002AD799519A11D8B444A80AD0800EBD2595
:10140000D96E020EBE21DA6E2E0EDF6EBD4BBE2BE4
:10141000800EBD25D96E020EBE21DA6E000EDF6E83
:10142000650EAB19D8A44AD4000EB66F4F0EB56F37
:10143000800EB525D96E020EB621DA6E000EDF6E73
:10144000000EA66F000EA56FBCAF08D0000EA66FF1
:10145000010EA56FBB6DBC1FD8B0BC2B000EA86FD2
:10146000020EA76F2AD0B507D8A0B607800EB52503
:10147000D96E020EB621DA6EBBC011F0BCC012F0FC
:10148000000E146E0A0E136E4EECAAF01150300FBF
:10149000DF6EBBC011F0BCC012F0000E146E0A0E5D
:1014A000136E5FECA8F011C0BBF012C0BCF0A70730
:1014B000D8A0A807A907D8A0AA07BB51BC11D8A4D7
:1014C000D2D7A8BF05D0A851CEE1A705D8B0CBD7B9
:1014D000B507D8A0B607A551A611D8A404D0000E10
:1014E000946F2B0E03D0000E946F2D0E936F800E11
:1014F000B525D96E020EB621DA6E60004FF2DFFF1D
:10150000A907D8A0AA07B507D8A0B607BF0E8C6F49
:10151000FF0E8D6F8B518E6F8F6B8C518E278D517F
:101520008F238F5104E11A0E8E5DD8A004D0000ED7
:10153000966F650E03D0000E966F450E956F800E68
:10154000B525D96E020EB621DA6E600057F2DFFFC4
:10155000A907D8A0AA07800EBD25156E020EBE21D0
:10156000166E800EB525176E020EB621186E1FEC92
:10157000ACF05EEF86F0600E3901D96F000EDB6FC4
:10158000000EDD6F080EDF6F000EDE6F3AECADF07F
:10159000B6ECB2F021ECB3F03AECB3F0A8ECB2F058
:1015A000000E0101B76F000E4D6E000E4C6E000E66
:1015B0004C24D96E040E4D20DA6E000EDF6E4C4ABC
:1015C0004D2A4D5004E1800E4C5CD8A0F0D7000E9F
:1015D0004D6E000E4C6E700E4C24D96E030E4D20D5
:1015E000DA6E000EDF6E4C4A4D2A4D5004E1800E3B
:1015F0004C5CD8A0F0D7000E4D6E000E4C6E000E65
:101600004C24D96E020E4D20DA6E000EDF6E4C4A6D
:101610004D2A4D5004E17F0E4C5CD8A0F0D7000E4F
:101620004D6E000E4C6EC10E4C24D96E010E4D2035
:10163000DA6E000EDF6E4C4A4D2A4D5004E1090E61
:101640004C5CD8A0F0D7000E486E040E496E37EC03
:10165000AFF0F1ECA4F0000E4D6E000E4C6EBA88A7
:10166000110E0201F76F3C0EF66FCB0EE82EFED77F
:10167000F62FFCD7F72FFAD7BA98110E0201F76FA1
:101680003C0EF66FCB0EE82EFED7F62FFCD7F72FC9
:10169000FAD74C4A4D2A4D5004E1080E4C5CD8A0B4
:1016A000DED7BA88ACECAEF0090E0201F76F1E0E61
:1016B000F66FE40EE82EFED7F62FFCD7F72FFAD7F9
:1016C00000F014ECB3F014ECB3F0DA0E116EFE0E71
:1016D000126E17ECAFF0000E4D6E000E4C6ED890EF
:1016E0004C34D96E4D34DA6ED00ED926020EDA2281
:1016F0006F0078FF11F06F0074FF12F017ECAFF07D
:101700004C4A4D2A4D5004E1090E4C5CD8A0E7D755
:1017100014ECB3F048C0EAF149C0EBF1840E0101CA
:10172000EC6FFB0EED6F920EEE6FFF0EEF6FB50ECE
:10173000F06FFF0EF16F090EF36F380EF26F68EC69
:10174000ADF048C011F049C012F061ECAEF014ECFD
:10175000B3F0000E126E020E116E23ECB0F0BA0E52
:10176000116EFD0E126E17ECAFF025ECB2F0FF0E0D
:10177000116EFB0E126E17ECAFF0FBEC97F014EC51
:10178000B3F0D40E116EF90E126E17ECAFF0270EF7
:101790000001FF6F000E4F6E140E4E6E000E010121
:1017A000EA6F020EEB6F6C0EEC6FFC0EED6FFFC07C
:1017B000EEF1EF6BFFC0F0F1F16B68ECADF0000EF5
:1017C000116E020E126E61ECAEF03D017589CD0E08
:1017D000116EFA0E126E17ECAFF03D01738F4EECE6
:1017E000A0F014ECB3F0010E1CECA8F0070E116E83
:1017F000FA0E126E17ECAFF021ECB3F03AECB3F046
:1018000014ECB3F0000E0101866F000E856FE70E39
:10181000116EFC0E126E17ECAFF0CA0E116EFC0EBC
:10182000126E17ECAFF014ECB3F0010E1CECA8F044
:10183000020E1CECA8F0000E0101D46F010ED36F54
:1018400046C011F047C012F0136A146A000EAEECE5
:101850009FF011C038F012C039F013C03AF014C034
:101860003BF0330E3C6E330E3D6E230E3E6E410E4A
:101870003F6EB6EC96F038C066F139C067F13AC0F9
:1018800068F13BC069F146C011F047C012F071EC3D
:10189000B0F0000E0101EA6F020EEB6FE60EEC6F86
:1018A000FD0EED6F46C0EEF147C0EFF166C1F0F1FD
:1018B00067C1F1F168C1F2F169C1F3F1000EF56F92
:1018C000250EF46F68ECADF0010E386E000E396E27
:1018D000020E3A6E010EEDECB2F0000E0101D46F73
:1018E000020ED36F8FC111F090C112F0136A146A07
:1018F000000EAEEC9FF011C038F012C039F013C0EA
:101900003AF014C03BF0330E3C6E330E3D6E230EA6
:101910003E6E410E3F6EB6EC96F038C062F139C0B3
:1019200063F13AC064F13BC065F18FC111F090C121
:1019300012F071ECB0F0000E0101EA6F020EEB6FD5
:10194000D00EEC6FFD0EED6F8FC1EEF190C1EFF197
:1019500062C1F0F163C1F1F164C1F2F165C1F3F16B
:10196000000EF56F250EF46F68ECADF0010E386EC9
:10197000000E396E020E3A6E020EEDECB2F0000E61
:10198000126E030E116E23ECB0F0010E1CECA8F0E9
:10199000020E1CECA8F06D0E116EF80E126E17EC14
:1019A000AFF0C5EC91F00F0E116EFF0E126E17EC3A
:1019B000AFF095ECADF0000E0401006F000E486E24
:1019C000040E496EC4803A016681000E656F000EF8
:1019D000676F6791C382000E556F55935683579377
:1019E000000E576F000E0101766F000E756F000E2E
:1019F000AD6FE10E116EF70E126E17ECAFF0670EC1
:101A0000116EF90E126E17ECAFF0280E116EF80E73
:101A1000126E17ECAFF0550E116EFD0E126E17EC34
:101A2000AFF0CFECAFF03901908FD28CD28ED28E46
:101A3000000E486E040E496ED70E116EFB0E126E2C
:101A400017ECAFF0A20E116EFE0E126E17ECAFF097
:101A500056ECAFF014ECB2F02E0E50ECB3F0090ED1
:101A60000201F76F1E0EF66FE40EE82EFED7F62F7A
:101A7000FCD7F72FFAD700F00101885104E1090ED5
:101A8000875DD8A0E9D7010E55ECA6F04A0E116E7D
:101A9000FC0E126E17ECAFF014ECB3F06DECB3F07B
:101AA0000101B46F000E9A6F000E996F000E7E6FE9
:101AB000000E7D6F14ECB2F07FECACF0000E020172
:101AC000006F000E0101EA6F020EEB6F310EEC6F3A
:101AD000FF0EED6F99C1EEF19AC1EFF146C0F0F142
:101AE00047C0F1F168ECADF0010E386E000E396EB2
:101AF000020E3A6E010EEDECB2F0000E116E020E07
:101B0000126E61ECAEF0000E0201006F000E0101DA
:101B1000EA6F020EEB6F9E0EEC6FFF0EED6F8FC142
:101B2000EEF190C1EFF168ECADF0000E116E020E17
:101B3000126E61ECAEF0010E386E000E396E020EC0
:101B40003A6E020EEDECB2F0000E0101866F010E4E
:101B5000856FFBEC9CF079C111F07AC112F0136A29
:101B6000146A000EAEEC9FF011C01FF012C020F0FE
:101B700013C021F014C022F00A0E236ED70E246E7B
:101B8000A30E256E3A0E266E88EC93F01FC03EF130
:101B900020C03FF121C040F122C041F17BC111F0D2
:101BA0007CC112F0000E12BEFF0E136E146E010EF9
:101BB000AEEC9FF011C01FF012C020F013C021F056
:101BC00014C022F06F0E236E120E246E830E256E4B
:101BD000390E266E88EC93F01FC042F120C043F10D
:101BE00021C044F122C045F1000E0101EA6F020E4E
:101BF000EB6F270EEC6FFE0EED6F3EC1EEF13FC1B5
:101C0000EFF140C1F0F141C1F1F142C1F2F143C144
:101C1000F3F144C1F4F145C1F5F168ECADF0000E0B
:101C2000116E020E126E61ECAEF0010E386E000EF7
:101C3000396E020E3A6E030EEDECB2F0000E0101A9
:101C4000EA6F020EEB6F520EEC6FFF0EED6F3AC1B2
:101C5000EEF13BC1EFF13CC1F0F13DC1F1F168ECB7
:101C6000ADF0000E116E020E126E61ECAEF0010EC0
:101C7000386E000E396E020E3A6E040EEDECB2F0C4
:101C800014ECB3F0BA78000E4D6E000E4C6E0101EC
:101C9000AF51D8B465D00F0E266E220E5AECABF0C1
:101CA0000101B36F110E266E220E5AECABF001014A
:101CB000B26F6DECB3F00101B46F000EEA6F020E6B
:101CC000EB6F2A0EEC6FFB0EED6FCBC111F0CCC1A8
:101CD00012F0CDC113F0CEC114F0E80E156E030E54
:101CE000166E000E176E000E186EA1ECA8F011C053
:101CF000EEF112C0EFF113C0F0F114C0F1F1CBC15D
:101D000011F0CCC112F0CDC113F0CEC114F0E80E29
:101D1000156E030E166E000E176E000E186EF4ECA4
:101D2000AAF011C0F2F112C0F3F113C0F4F114C023
:101D3000F5F1B2C1F6F1F76BB3C1F8F1F96B68ECEC
:101D4000ADF0000E116E020E126E61ECAEF014ECEE
:101D5000B3F0000E0101AF6F000E4D6EFA0E4C6E27
:101D60002A0E0201F66F8D0EE82EFED7F62FFCD755
:101D700000D04C4A4D2A4D5004E1FA0E4C5CD8A0DC
:101D800086D70101BC05D8B4CDEC8EF0994B9A2BC7
:101D9000000E7E6F000E7D6F8FD6BC05D8A412009A
:101DA000CD0E116EFF0E126E17ECAFF0700E116EAD
:101DB000030E126E61ECAEF014ECB3F0700E010184
:101DC000956F030E966F600057F6D9FF60005BF6C3
:101DD000DAFF480EDE18D8A43BD020EE01F0955172
:101DE000D9269651DA22650EDE18D8A431D020EE1D
:101DF00002F09551D9269651DA226C0EDE18D8A43D
:101E000027D020EE03F09551D9269651DA22700E94
:101E1000DE18D8A41DD0C60E116EFF0E126E17EC80
:101E2000AFF0AF0E116EFB0E126E17ECAFF02B0E73
:101E3000116EF90E126E17ECAFF0EF0E116EF80E78
:101E4000126E17ECAFF0000E0101956F000E966F49
:101E5000600057F6D9FF60005BF6DAFF520EDE181D
:101E6000D8A42DD020EE01F09551D9269651DA2232
:101E7000650EDE18D8A423D020EE05F09551D926A2
:101E80009651DA22720EDE18D8A419D020EE06F090
:101E90009551D9269651DA22740EDE18D8A40FD0A7
:101EA000000EAD6FBA86890E116EFD0E126E17EC24
:101EB000AFF0BA88000E0101956F000E966F6000BA
:101EC00057F6D9FF60005BF6DAFF500EDE18D8A493
:101ED00019D220EE01F09551D9269651DA22570EEB
:101EE000DE18D8A40FD220EE02F09551D9269651D3
:101EF000DA224D0EDE18D8A405D220EE04F095515A
:101F0000D9269651DA223D0EDE18D8A4FBD120EE58
:101F100003F09551D9269651DA22DF500001FE6F69
:101F2000000E01019E6F000E9D6FD00EFA6FFF0E26
:101F3000FB6F0001FE510101FC6FFD6BFA51FC27A4
:101F4000FB51FD23FD5103E10A0EFC5DD8B0D5D154
:101F5000300E0001FE65D1D1330EFE61CED10101FC
:101F60009D4B9E2BD00EFA6FFF0EFB6F20EE05F0FF
:101F70009551D9269651DA22DF50FC6FFD6BFA514C
:101F8000FC27FB51FD23FD511FE10A0EFC5DD8B07B
:101F90001BD020EE05F09551D9269651DA22DF505C
:101FA000FA6FD00EFA25116E126AFF0E1222030E7E
:101FB000146EE80E136EC5ECB1F011C0D3F112C06F
:101FC000D4F101019D4B9E2BD00EFA6FFF0EFB6FDB
:101FD00020EE06F09551D9269651DA22DF50FC6F9B
:101FE000FD6BFA51FC27FB51FD23FD5120E10A0E48
:101FF000FC5DD8B01CD020EE06F09551D926965144
:10200000DA22DF50FA6FFA51640D6F00CCFFFBF15A
:102010006F00D0FFFCF1D351FB27D451FC23400EBD
:10202000FB25D36FED0EFC21D46F9D4B9E2BD00E64
:10203000FA6FFF0EFB6F20EE07F09551D9269651EF
:10204000DA22DF50FC6FFD6BFA51FC27FB51FD23B8
:10205000FD5120E10A0EFC5DD8B01CD020EE07F047
:102060009551D9269651DA22DF50FA6FFA510A0DAE
:102070006F00CCFFFBF16F00D0FFFCF1D351FB27C9
:10208000D451FC23200EFB25D36FFE0EFC21D46F10
:102090009D4B9E2BD00EFA6FFF0EFB6F20EE08F0CB
:1020A0009551D9269651DA22DF50FC6FFD6BFA511B
:1020B000FC27FB51FD23FD511AE10A0EFC5DD8B04F
:1020C00016D020EE08F09551D9269651DA22DF502D
:1020D000FA6FFA51D325FB6F000ED421FC6FD00E9E
:1020E000FB25D36FFF0EFC21D46F9D4B9E2B050E5D
:1020F0009D199E11D8A4E4D0F80ED35D030ED459D7
:10210000D8B0DED0BC8AB4D07A0E116EFF0E126E3B
:1021100017ECAFF0D3C146F0D4C147F0D3C111F0F2
:10212000D4C112F0136A146A000EAEEC9FF011C015
:1021300038F012C039F013C03AF014C03BF0330E3F
:102140003C6E330E3D6E230E3E6E410E3F6EB6EC7E
:1021500096F038C066F139C067F13AC068F13BC00B
:1021600069F1000E0101EA6F020EEB6F510EEC6F88
:10217000FE0EED6F46C0EEF147C0EFF166C1F0F123
:1021800067C1F1F168C1F2F169C1F3F1000EF56FB9
:10219000250EF46F68ECADF0010E386E000E396E4E
:1021A000020E3A6E010EEDECB2F046C011F047C0DF
:1021B00012F071ECB0F06DD0D3C18FF1D4C190F1B9
:1021C000D3C111F0D4C112F0136A146A000EAEEC40
:1021D0009FF011C038F012C039F013C03AF014C0AB
:1021E0003BF0330E3C6E330E3D6E230E3E6E410EC1
:1021F0003F6EB6EC96F038C062F139C063F13AC078
:1022000064F13BC065F1000E0101EA6F020EEB6F55
:102210003C0EEC6FFE0EED6F8FC1EEF190C1EFF151
:1022200062C1F0F163C1F1F164C1F2F165C1F3F192
:10223000000EF56F250EF46F68ECADF0010E386EF0
:10224000000E396E020E3A6E020EEDECB2F08FC146
:1022500011F090C112F057ECB0F01BD0000E00014D
:10226000FE6F600E116EFF0E126E17ECAFF011D004
:102270000001FE510101FA6FFB6BFB51000AD8A46B
:10228000EDD7FA51310AD8B43FD7030AD8B494D75E
:10229000E5D70001FE51D8B411D0000E116E020E28
:1022A000126E61ECAEF014ECB3F0D00E0101FA6FD7
:1022B000C90EE82EFED7FA2FFCD700D0BC9A1DD04D
:1022C000000EEA6F020EEB6F6C0EEC6FFA0EED6F04
:1022D000FEC0EEF1EF6BD3C1F0F1D4C1F1F168ECC7
:1022E000ADF0000E116E020E126E61ECAEF08D0EAE
:1022F000116EF70E126E17ECAFF0000E0101956F24
:10230000000E966F600057F6D9FF60005BF6DAFFAB
:102310004D0EDE18D8A436D020EE01F09551D92606
:102320009651DA22410EDE18D8A42CD020EE02F00D
:102330009551D9269651DA223D0EDE18D8A422D026
:1023400020EE03F09551D9269651DA22DF50000194
:10235000FE6F310EFE19D8A408D0BA86FE0E116E9B
:10236000FE0E126E17ECAFF008D0C80E116EFE0E06
:10237000126E17ECAFF0BA96BA88000E0101956F95
:10238000000E966F000EBC6F12009D0E116EFA0EBD
:10239000126E17ECAFF0C10E0101936F010E946F36
:1023A000000EC16F470EC26F3F0EC36F400E00019B
:1023B000FF6F030EFE6F93C126F094C127F0FEC09D
:1023C00028F0296AFF5187ECAEF0B10E116EF80EBD
:1023D000126E17ECAFF0050E0101C16F000EC26F57
:1023E000140EC36F400E0001FF6FC10E0101936F09
:1023F000010E946F030E0001FE6F93C126F094C18D
:1024000027F0FEC028F0296AFF5187ECAEF03A0EA3
:10241000116EFA0E126E17ECAFF0060E0101C16FCD
:10242000800EC26F000EC36F400E0001FF6FC10E21
:102430000101936F010E946F030E0001FE6F93C1B3
:1024400026F094C127F0FEC028F0296AFF5187ECDE
:10245000AEF09F0E116EF90E126E17ECAFF0070E74
:102460000101C16F090EC26F600EC36F400E000103
:10247000FF6FC10E0101936F010E946F030E0001F7
:10248000FE6F93C126F094C127F0FEC028F0296AA0
:10249000FF5187ECAEF0400E0001FF6F000E01010E
:1024A000C16F000EC26FC10E936F010E946F040EC8
:1024B000266E93C127F094C128F0000E2A6E030EF9
:1024C000296E0001FF51BDECAAF00101C1510001CC
:1024D000FD6FFC6B0101C2510001FC250101D36FAE
:1024E000000E0001FD210101D46F000EEA6F020E03
:1024F000EB6FAC0EEC6FFC0EED6FD3C1EEF1D4C1FF
:10250000EFF168ECADF0000E116E020E126E61EC90
:10251000AEF0400E0001FF6F000E0101C16F000E12
:10252000C26FC10E936F010E946F070E266E93C19A
:1025300027F094C128F0000E2A6E030E296E0001C8
:10254000FF51BDECAAF00101C1510001FD6FFC6B10
:102550000101C2510001FC250101D36F000E0001F1
:10256000FD210101D46F6F0E236E120E246E030E37
:10257000256E410E266ED3C111F0D4C112F0136A3C
:10258000146A000EAEEC9FF011C01FF012C020F0D4
:1025900013C021F014C022F088EC93F01FC038F073
:1025A00020C039F021C03AF022C03BF0000E3C6E52
:1025B000000E3D6E000E3E6E470E3F6EB6EC96F07E
:1025C00038C03AF139C03BF13AC03CF13BC03DF173
:1025D000000E0101EA6F020EEB6F8C0EEC6FFC0E29
:1025E000ED6F3AC1EEF13BC1EFF13CC1F0F13DC1FD
:1025F000F1F168ECADF0000E116E020E126E61EC9E
:10260000AEF0400E0001FF6F000E0101C16F000E21
:10261000C26F000EC36FC10E936F010E946FFE0E5A
:10262000266E93C127F094C128F0000E2A6E030E87
:10263000296E0001FF51BDECAAF00101C15100015A
:10264000FD6FFC6B0101C2510001FC250101D36F3C
:10265000000E0001FD210101D46F000EEA6F020E91
:10266000EB6F200EEC6FFD0EED6FD3C1EEF1D4C118
:10267000EFF168ECADF0000E116E020E126E61EC1F
:10268000AEF0400E0001FF6F000E0101C16F000EA1
:10269000C26F000EC36FC10E936F010E946FFF0ED9
:1026A000266E93C127F094C128F0000E2A6E030E07
:1026B000296E0001FF51BDECAAF00101C1510001DA
:1026C000FD6FFC6B0101C2510001FC250101D36FBC
:1026D000000E0001FD210101D46F000EEA6F020E11
:1026E000EB6F3B0EEC6FFD0EED6FD3C1EEF1D4C17D
:1026F000EFF168ECADF0000E116E020E126E61EC9F
:10270000AEF0250E116EFC0E126E17ECAFF012003B
:102710002250800B2B6E225022242D6E21BE2D8044
:102720002D50D8B40DD02D28D8A408D0000E1F6E7F
:10273000000E206E000E216E000E226E218E08D03B
:10274000000E1F6E000E206E000E216E000E226E17
:102750002650800B2B1A265026242C6E25BE2C804A
:102760002C50D8B40DD02C28D8A408D0000E236E3D
:10277000000E246E000E256E000E266E258E08D0EB
:10278000000E236E000E246E000E256E000E266EC7
:102790002C50D8B403D02D50D8A409D0000E1F6EF1
:1027A000000E206E000E216E000E226E12002550CB
:1027B0001F026F00CCFF36F06F00D0FF37F03650AD
:1027C0002E6E2F6A306A316A3750326E336A346A3D
:1027D000356A245020026F00CCFF36F06F00D0FF26
:1027E00037F036502E26000E2F223022312237505D
:1027F0003226000E332234223522235021026F006C
:10280000CCFF36F06F00D0FF37F036502E26000E8A
:102810002F223022312237503226000E332234222A
:10282000352230C031F02FC030F02EC02FF02E6A8C
:10283000235020026F00CCFF36F06F00D0FF37F03E
:1028400036502E2637502F22000E3022000E312215
:1028500024501F026F00CCFF36F06F00D0FF37F01E
:1028600036502E2637502F22000E3022000E3122F5
:1028700030C031F02FC030F02EC02FF02E6A235020
:102880001F026F00CCFF36F06F00D0FF37F03650DC
:102890002E2637502F22000E3022000E31222550D6
:1028A00020026F00CCFF36F06F00D0FF37F03650BB
:1028B000322637503322000E3422000E35222450A7
:1028C00021026F00CCFF36F06F00D0FF37F036509A
:1028D000322637503322000E3422000E3522255086
:1028E00021026F00CCFF36F06F00D0FF37F036507A
:1028F000276E3750286E296A2A6A29C02AF028C014
:1029000029F027C028F0276A275032262850332282
:10291000295034222A50352231503226000E3322DB
:102920003422352230C031F02FC030F02EC02FF0CD
:102930002E6A2C502DC027F0286A2726000E282248
:10294000820E2724366EFF0E2820376E0FD0D890C7
:10295000323633363436353631BE3280D8902E3664
:102960002F36303631363606D8A0370634AEEFD79C
:10297000000E2C6E31AE17D0FF0E2E14276EFF0EF8
:102980002F14286EFF0E3014296E7F0E31142A6E1C
:102990002750281029102A10D8B403D0010E2C6E0D
:1029A00002D032B0FBD72C50D8B41FD0010E322643
:1029B000000E33223422352235A017D032C027F042
:1029C00033C028F034C029F035C02AF02A342A3226
:1029D00029322832273227C032F028C033F029C0EC
:1029E00034F02AC035F0364A372A37BE0DD037507A
:1029F00003E13628D8A008D0000E326E000E336EE8
:102A0000800E346E7F0E20D037BE05D037500EE1D9
:102A10003604D8B00BD0000E326E000E336E000EAE
:102A2000346E000E356E000E2B6E0FD036C02DF0BA
:102A3000FF0E3216FF0E33167F0E3416000E3516BB
:102A40002DB0348ED8902D30356E2B50351232C0CB
:102A50001FF033C020F034C021F035C022F0120046
:102A60001450800B1D6E145014241F6E13BE1F8053
:102A70001F50D8B40DD01F28D8A408D0000E116E56
:102A8000000E126E000E136E000E146E138E06D022
:102A9000000E116E000E126E000E136E000E146EFC
:102AA0001850800B1E6E1D501E18D8A41D8C185077
:102AB00018241E6E17BE1E801E50D8B40DD01E28BE
:102AC000D8A408D0000E156E000E166E000E176EFC
:102AD000000E186E178E06D0000E156E000E166EC4
:102AE000000E176E000E186E1F501E5CD8B022D05C
:102AF0001DAC02D0800E1D1A1FC020F01EC01FF09A
:102B000020C01EF011C020F015C011F020C015F03B
:102B100012C020F016C012F020C016F013C020F032
:102B200017C013F020C017F014C020F018C014F024
:102B300020C018F0000E206E1F501EC019F01A6A37
:102B4000195E000E1A5A1ABE2CD01A5004E11A0E41
:102B5000195CD8A026D01150121013101410D8B43C
:102B600002D0010E01D0000E206E000E116E000E7C
:102B7000126E000E136E000E146E1EC01FF015D0E4
:102B800020A005D0D89020300109206E02D0D89026
:102B9000203211B0208E143414321332123211321A
:102BA0001F2A1E501F5CD8A0EBD71DBC28D01F5079
:102BB000D8A409D0000E116E000E126E000E136E16
:102BC000000E146E120015501126165012221750C6
:102BD00013221850142214A071D020A005D0D89030
:102BE00020300109206E02D0D890203211B0208E02
:102BF000143414321332123211321F2A5FD015509E
:102C0000115C16501258175013581450800A196E40
:102C10001850800A1958D8B025D01150155C196E7B
:102C2000125016581A6E135017581B6E145018581D
:102C30001C6EFF0E1924116EFF0E1A20126EFF0E6D
:102C40001B20136EFF0E1C20146E800E1D1A206CAC
:102C50002050D8A40FD0010E1126000E12221322EC
:102C6000142208D01550115E1650125A1750135ADC
:102C70001850145A1150121013101410D8A41CD04C
:102C80002050D8A419D0000E116E000E126E000E46
:102C9000136E000E146E1200D890113612361336D1
:102CA000143620BE118020A002D0D88001D0D89048
:102CB00020361F50D8A41F0613AEEED7000E1E6E8E
:102CC00020AE0BD020C019F07F0E1916D8B403D057
:102CD000010E1E6E02D011B0FBD71E50D8B420D00A
:102CE000010E1126000E12221322142214A018D055
:102CF00011C019F012C01AF013C01BF014C01CF060
:102D00001C341C321B321A32193219C011F01AC08D
:102D100012F01BC013F01CC014F01F28D8A41F2AE7
:102D20001F28D8B403D01F50D8A40DD0000E116EA8
:102D3000000E126E000E136E000E146E1F50D8A4FB
:102D400002D0000E1D6E1FA002D0138E01D0139E64
:102D5000D8901F30146E1DBE148E11C011F012C019
:102D600012F013C013F014C014F012003B50800B8B
:102D70000001686F3B503B246F6F3ABE6F816F510B
:102D8000D8B40DD06F29D8A408D0000E386E000E2C
:102D9000396E000E3A6E000E3B6E3A8E06D0000E73
:102DA000386E000E396E000E3A6E000E3B6E3F50CC
:102DB000800B681B3F503F24706F3EBE7081705186
:102DC000D8B40DD07029D8A408D0000E3C6E000EE7
:102DD0003D6E000E3E6E000E3F6E3E8E06D0000E23
:102DE0003C6E000E3D6E000E3E6E000E3F6E3C507F
:102DF0003D103E103F10D8A417D0000E386E000EC4
:102E0000396E000E3A6E000E3B6E800E3A127F0E47
:102E10003B1268513B1238C038F039C039F03AC023
:102E20003AF03BC03BF012006F51D8A409D0000E1D
:102E3000386E000E396E000E3A6E000E3B6E1200B8
:102E400070516FC060F0616B605F000E615B7F0E60
:102E50006025696F000E61216A6F38C064F039C067
:102E600065F03AC066F03BC067F0000E386E000EA9
:102E7000396E000E3A6E000E3B6E000E6B6F000E48
:102E80006C6F000E6D6F000E6E6F000E706F28D0AD
:102E90007051D8B411D0D89064376537663767372A
:102EA000D890383639363A363B366EBF3880D890AF
:102EB0006B376C376D376E373C50645D3D506559EC
:102EC0003E5066593F506759D8A009D06E8D3C508E
:102ED000645F3D50655B3E50665B3F50675B702BA7
:102EE000190E7065D5D76451651166116711D8B494
:102EF00011D06B810FD0D890383639363A363B3600
:102F00006EBF3880D8906B376C376D376E37690776
:102F1000D8A06A073AAEEFD7000E706F6EAF17D029
:102F2000FF0E6B15606FFF0E6C15616FFF0E6D1558
:102F3000626F7F0E6E15636F6051611162116311D4
:102F4000D8B403D0010E706F02D038B0FBD77051E7
:102F5000D8B41FD0010E3826000E39223A223B2267
:102F60003BA017D038C060F039C061F03AC062F0C1
:102F70003BC063F06335633362336133603360C0F9
:102F800038F061C039F062C03AF063C03BF0694B81
:102F90006A2B6ABF10D06A5103E16929D8A00BD00F
:102FA000000E6A6F6969000E386E000E396E000EF1
:102FB0003A6E000E3B6E6ABF05D06A5111E1690599
:102FC000D8B00ED0000E6A6F000E696F000E386E1A
:102FD000000E396E000E3A6E000E3B6E000E686FEA
:102FE00069C06FF06FA102D03A8E01D03A9ED8909E
:102FF0006F313B6E0ED7000E486E040E496E6000B6
:1030000023F1D9FF600027F1DAFF000EDF6E3D01EA
:103010007599738F000E0101FD6F020EFC6FFCC1EC
:1030200011F0FDC112F069ECB2F00009D8B4F6D08D
:103030000101FD35FD310001FC6F0101FC31D36F51
:10304000FCC0D4F148C0EAF149C0EBF1FC0EEC6FD2
:10305000FA0EED6FFCC1EEF1FDC1EFF1D3C1F0F15D
:10306000D4C1F1F168ECADF090D048C01FF049C078
:1030700020F0A20E216EFD0E226E01ECB2F0C6D041
:1030800048C01FF049C020F06F0E216EFD0E226E69
:1030900001ECB2F0BBD0000E116E020E126E200ECB
:1030A000136EFF0E146E27ECABF048C011F049C050
:1030B00012F03BECAEF011C0FAF112C0FBF10101CD
:1030C000FA514824156EFB514920166E000E176EFA
:1030D000020E186E1FECACF099D048C01FF049C02A
:1030E00020F0EC0E216EFE0E226E01ECB2F08ED0BE
:1030F00048C01FF049C020F0B50E216EFE0E226EB2
:1031000001ECB2F083D048C01FF049C020F06D0E32
:10311000216EFF0E226E01ECB2F078D048C01FF095
:1031200049C020F0FC0E216EFD0E226E01ECB2F0C3
:103130006DD048C01FF049C020F0420E216EFF0E36
:10314000226E01ECB2F062D048C01FF049C020F0FE
:10315000AA0E216EFF0E226E01ECB2F057D048C0CD
:103160001FF049C020F0040E216EFD0E226E01EC0E
:10317000B2F04CD048C01FF049C020F0860E216E3E
:10318000FF0E226E01ECB2F041D0D3C1FCF0D4C1ED
:10319000FDF00001FD51000AD8A4ECD7FC51200A33
:1031A000D8B463D7010AD8B460D7030AD8B45DD7BE
:1031B000010AD8B45AD7040AD8B462D70F0AD8B4CF
:1031C0006AD7010AD8B467D7030AD8B464D71D0AEE
:1031D000D8B483D70F0AD8B48BD7010AD8B488D70C
:1031E000030AD8B485D7010AD8B482D7070AD8B45D
:1031F0008AD77C0AD8B492D7170AD8B49AD73F0A8C
:10320000D8B4A2D7C80AD8B4AAD7B4D748C011F046
:1032100049C012F061ECAEF014ECB3F0020E010103
:10322000FC25FC6F000EFD21FD6FFDBFF8D6FD51A2
:1032300004E1FC0EFC5DD8A0F2D63D01739F7589B8
:1032400014ECB3F0738F12002EC068F02FC069F039
:1032500030C06AF031C06BF032C06CF033C06DF03A
:1032600034C06EF035C06FF06FAF02D0010E01D0E8
:10327000000E666F676B66516711D8B410D06F1F70
:103280006E1F6D1F6C1F6B1F6A1F691F686D000E1C
:1032900069236A236B236C236D236E236F2343AE54
:1032A000449243BE05D0435008E14204D8B005D053
:1032B000000E636F010E626F04D042C062F043C023
:1032C00063F040C064F041C065F066516711D8A456
:1032D00002D044A403D06407D8A06507000E716F24
:1032E0004F0E706F000E0201CF6F7CD07007D8A018
:1032F0007107800E7025D96E020E7121DA6E68C0DA
:1033000011F069C012F06AC013F06BC014F06CC009
:1033100015F06DC016F06EC017F06FC018F00A0EF1
:10332000196E000E1A6E000E1B6E000E1C6E000E43
:103330001D6E000E1E6E000E1F6E000E206EE9EC5C
:10334000A0F011C036F012C037F013C038F014C02E
:1033500039F015C03AF016C03BF017C03CF018C069
:103360003DF036C023F038C024F0BFECB0F023505D
:10337000300FDF6E6207D8A063076407D8A0650727
:1033800068C011F069C012F06AC013F06BC014F08D
:103390006CC015F06DC016F06EC017F06FC018F05D
:1033A0000A0E196E000E1A6E000E1B6E000E1C6EB9
:1033B000000E1D6E000E1E6E000E1F6E000E206EA3
:1033C0006AEC9EF011C068F012C069F013C06AF098
:1033D00014C06BF015C06CF016C06DF017C06EF025
:1033E00018C06FF0000171BF1FD0715103E170056B
:1033F000D8A01AD0685169116A116B116C116D1146
:103400006E116F11D8A472D763BF05D0635102E16A
:103410006205D8B06BD765BF07D0655103E164057D
:10342000D8A002D044B262D766516711D8A402D0A6
:1034300044A418D07007D8A0710766516711D8A4AA
:1034400004D0000E616F2B0E03D0000E616F2D0EA5
:10345000606F800E7025D96E020E7121DA6E6000E9
:1034600083F1DFFF2CC021F02DC022F0800E7025EB
:10347000236E020E7121246E64C025F065C026F013
:103480008CECA7F021C02CF022C02DF0120043AE2E
:10349000449243BE05D0435008E14204D8B005D061
:1034A000000E616F010E606F04D042C060F043C037
:1034B00061F040C062F041C063F044A804D0FE0E49
:1034C0006227FF0E63232EC064F02FC065F030C06A
:1034D00066F031C067F032C068F033C069F034C0C4
:1034E0006AF035C06BF0000E6D6F4F0E6C6F000E02
:1034F0000201CF6F82D06C07D8A06D070F0E641544
:103500006E6F6F6B6FBF08D06F5104E10A0E6E5D76
:10351000D8A002D0570E01D0300E6E256E6F000E6F
:103520006F216F6FBF0E376EFF0E386E3650396EDB
:103530003A6A3750392638503A223A5022E11A0E68
:10354000395CD8B01ED09F0E376EFF0E386E200E3D
:103550006E11396E000E6F113A6E375039263850A1
:103560003A223A500EE11A0E395CD8B00AD06EC039
:1035700017F06FC018F0EBECAFF017C06EF018C08A
:103580006FF0800E6C25D96E020E6D21DA6E600030
:10359000BBF1DFFF6007D8A061076207D8A063070F
:1035A00064C037F065C038F066C039F067C03AF0E3
:1035B00068C03BF069C03CF06AC03DF06BC03EF0B3
:1035C000050E09D0D8903E323D323C323B323A3281
:1035D000393238323732E82EF5D737C064F038C088
:1035E00065F039C066F03AC067F03BC068F03CC097
:1035F00069F03DC06AF03EC06BF000016DBF20D0A5
:103600006D5104E1020E6C5DD8A01AD064516511B1
:1036100066116711681169116A116B11D8A46BD713
:1036200061BF05D0615102E16005D8B064D763BFC6
:1036300007D0635103E16205D8A002D044B25BD742
:1036400044A817D06C07D8A06D07800E6C25D96EE2
:10365000020E6D21DA6E6000DBF0DFFF6C07D8A090
:103660006D07800E6C25D96E020E6D21DA6E300E5C
:10367000DF6E2CC021F02DC022F0800E6C25236E51
:10368000020E6D21246E62C025F063C026F08CEC22
:10369000A7F021C02CF022C02DF0120043AE4492BE
:1036A00043BE05D0435008E14204D8B005D0000E17
:1036B000616F010E606F04D042C060F043C061F0E2
:1036C00040C062F041C063F02EC064F02FC065F0CE
:1036D00030C066F031C067F032C068F033C069F0C6
:1036E00034C06AF035C06BF0000E6D6F4F0E6C6F1A
:1036F000000E0201CF6F76D06C07D8A06D07800E48
:103700006C25D96E020E6D21DA6E64C011F065C0B1
:1037100012F066C013F067C014F068C015F069C0FD
:1037200016F06AC017F06BC018F00A0E196E000E82
:103730001A6E000E1B6E000E1C6E000E1D6E000E2B
:103740001E6E000E1F6E000E206EA7ECA5F011C0BD
:1037500036F012C037F013C038F014C039F015C07D
:103760003AF016C03BF017C03CF018C03DF03650A0
:10377000300FDF6E6007D8A061076207D8A063072B
:1037800064C011F065C012F066C013F067C014F099
:1037900068C015F069C016F06AC017F06BC018F069
:1037A0000A0E196E000E1A6E000E1B6E000E1C6EB5
:1037B000000E1D6E000E1E6E000E1F6E000E206E9F
:1037C000C7ECA3F011C064F012C065F013C066F03E
:1037D00014C067F015C068F016C069F017C06AF031
:1037E00018C06BF000016C516D11D8B41AD064513F
:1037F000651166116711681169116A116B11D8A4FE
:103800007BD761BF05D0615102E16005D8B074D7A4
:1038100063BF07D0635103E16205D8A002D044B270
:103820006BD72CC021F02DC022F0800E6C25236EAA
:10383000020E6D21246E62C025F063C026F08CEC70
:10384000A7F021C02CF022C02DF0120032C181F06F
:1038500033C182F034C183F035C184F071C081F08E
:1038600072C082F073C083F074C084F0810E756FF3
:10387000FF0E766F81C077F082C078F083C079F058
:1038800084C07AF0180E05D0D8907A337933783323
:103890007733E82EF9D7775175257F6F000E7621A3
:1038A000806F80BF0FD0805104E1170E7F5DD8A0DC
:1038B00009D071C071F072C072F073C073F074C03F
:1038C00074F0120080BF5CD07FC075F0FF0E766F81
:1038D000FF0E776F7F0E786F000E796F756701D0DE
:1038E00007D079357933783377337633752FF6D738
:1038F00076C07BF077C07CF078C07DF079C07EF038
:1039000000017B518115756F7C518215766F7D5159
:103910008315776F7E518415786F75517611771105
:103920007811D8B4C6D781C075F082C076F083C054
:1039300077F084C078F0200E05D0D89078337733B4
:1039400076337533E82EF9D77551D8B408D07B514A
:1039500081277C5182237D5183237E5184237B1DCB
:10396000756F7C1D766F7D1D776F7E1D786F75512D
:10397000811776518217775183177851841732D087
:1039800081C075F082C076F083C077F084C078F093
:10399000200E05D0D8907833773376337533E82E00
:1039A000F9D7756708D0000E816F000E826F000E88
:1039B000836F000E16D0D8908135756F8235766F83
:1039C0008335776F8435786F75517611771178115B
:1039D000D8B408D0000E816F000E826F800E836F06
:1039E000BF0E846F81C071F082C072F083C073F02B
:1039F00084C074F01200000EC16F000EC26FC10EC1
:103A0000936F010E946F020E266E93C127F094C13E
:103A100028F0000E2A6E030E296E400EBDECAAF0AF
:103A20000101C1510001726F716B0101C2510001AE
:103A300071250101796F000E0001722101017A6F79
:103A4000000EC16F000EC26FC10E936F010E946F16
:103A5000010E266E93C127F094C128F0000E2A6E45
:103A6000030E296E400EBDECAAF00101C151000108
:103A7000726F716B0101C2510001712501017B6FF1
:103A8000000E0001722101017C6F000EC16F000E5B
:103A9000C26FC10E936F010E946F070E266E93C115
:103AA00027F094C128F0000E2A6E030E296E400EF6
:103AB000BDECAAF00101C1510001726F716B0101EF
:103AC000C251000171250101D36F000E0001722166
:103AD0000101D46F6F0E236E120E246E030E256E3D
:103AE000410E266ED3C111F0D4C112F0136A146ACC
:103AF000000EAEEC9FF011C01FF012C020F013C0FA
:103B000021F014C022F088EC93F01FC038F020C0E0
:103B100039F021C03AF022C03BF0000E3C6E000E9E
:103B20003D6E000E3E6E470E3F6EB6EC96F038C00E
:103B30003AF139C03BF13AC03CF13BC03DF1000ED7
:103B40000101C16F000EC26FC10E936F010E946F21
:103B5000040E266E93C127F094C128F0000E2A6E41
:103B6000030E296E400EBDECAAF00101C151000107
:103B7000726F716B0101C251000171250101776FF4
:103B8000000E000172210101786F120020EED5F1C4
:103B900010EE1FF0060E6F006FFFE3FFE806FBE27A
:103BA0001CC02AF01DC02BF02A502B10D8A403D023
:103BB0001F0E2A6E2B6A2AC011F02BC012F03BECAC
:103BC000AEF011C02EF012C02FF042C02CF043C056
:103BD0002DF02DBE0ED02E502C5C2D50800A1E6E66
:103BE0002F50800A1E58D8B004D02CC02EF02DC003
:103BF0002FF02EC02CF02FC02DF040C028F041C077
:103C000029F044A00DD016D0000E126E200E116EB9
:103C10001AC013F01BC014F0FEECA5F02E4A2F2A98
:103C200028502E5C2F50800A1E6E2950800A1E5884
:103C3000D8A0EAD7000E276E000E266E23D06000B3
:103C4000ABF0F6FF6000AFF0F7FF000EF86E1F0E4E
:103C5000F76403D00800F55007D06F00DBFFE1FFE9
:103C60006F00DFFFE2FFE7501E6E1E50116E126AFA
:103C70001AC013F01BC014F0FEECA5F02A4A2B2A40
:103C8000264A272A2C50265C2750800A1E6E2D506B
:103C9000800A1E58D8A0D3D744B00DD016D0000E3D
:103CA000126E200E116E1AC013F01BC014F0FEEC41
:103CB000A5F02E4A2F2A28502E5C2F50800A1E6E07
:103CC0002950800A1E58D8A0EAD72EC01AF02FC05B
:103CD0001BF01200000E226E20AE12D0201E1F1EFE
:103CE0001E1E1D1E1C1E1B1E1A1E196C000E1A22E3
:103CF0001B221C221D221E221F222022010E226EA8
:103D000018AE12D0181E171E161E151E141E131ED6
:103D1000121E116C000E12221322142215221622DA
:103D200017221822010E221A20EE23F0070EDE6A57
:103D3000E806FDE219501A101B101C101D101E1071
:103D40001F102010D8B446D0010E216E0AD0D89092
:103D500019361A361B361C361D361E361F362036CF
:103D6000212A20AEF4D7D89023362436253626369D
:103D70002736283629362A361950115C1A5012581F
:103D80001B5013581C5014581D5015581E501658CF
:103D90001F50175820501858D8A011D01950115E34
:103DA0001A50125A1B50135A1C50145A1D50155AAF
:103DB0001E50165A1F50175A2050185A2380D89058
:103DC00020321F321E321D321C321B321A3219327F
:103DD000212EC9D72250D8B410D02A1E291E281E41
:103DE000271E261E251E241E236C000E242225229B
:103DF00026222722282229222A2223C011F024C089
:103E000012F025C013F026C014F027C015F028C00A
:103E100016F029C017F02AC018F01200000E216E0B
:103E2000000E206E000E1F6E000E1E6E02D0184A8D
:103E3000192A600063F0F6FF600067F0F7FF000EDC
:103E4000F86E0800F550200AD8B4F1D7F70E1A6EB4
:103E5000FF0E1B6E600063F0F6FF600067F0F7FF77
:103E6000000EF86E0800F5501C6E1D6A1A501C26D4
:103E70001B501D221D500CE1050E1C5CD8B008D053
:103E8000D6D7000E1F6E010E1E6E184A192A36D0A4
:103E9000600063F0F6FF600067F0F7FF000EF86E59
:103EA0000800F5501A6E1B6A1B50000AD8A426D0D1
:103EB0001A502B0AD8B4E9D7060AD8B4E2D71ED0D4
:103EC00020C011F021C012F0000E146E0A0E136E05
:103ED000C5ECB1F0600063F0F6FF600067F0F7FF3B
:103EE000000EF86E0800F550115E000E125A300EEA
:103EF0001124206E000E1220216EC7D7D00E1A6E2C
:103F0000FF0E1B6E600063F0F6FF600067F0F7FFC6
:103F1000000EF86E0800F5501C6E1D6A1A501C2623
:103F20001B501D221D5004E10A0E1C5CD8A0C8D7EE
:103F30001E501F10D8A40DD020C01AF021C01BF0B5
:103F40001A1E1B1E1A4A1B2A1AC018F01BC019F091
:103F5000120020C018F021C019F01200196E19507B
:103F6000D8A414AE1AD011C015F012C016F013C0A8
:103F700017F014C018F0151E161E171E181E152A4D
:103F8000000E16221722182215C01BF016C01CF0B6
:103F900017C01DF018C01EF008D011C01BF012C0D1
:103FA0001CF013C01DF014C01EF01150121013109D
:103FB0001410D8A409D0000E116E000E126E000E5F
:103FC000136E000E146E1200960E1A6E06D01A2A88
:103FD000D8901E321D321C321B32000E1B14156E7F
:103FE000000E1C14166E000E1D14176EFE0E1E140D
:103FF000186E1550161017101810D8B40DD0E7D73A
:104000001A2A010E1B26000E1C221D221E22D890E9
:104010001E321D321C321B32000E1B14156E000E98
:104020001C14166E000E1D14176EFF0E1E14186E53
:104030001550161017101810D8B407D0E1D71A066B
:10404000D8901B361C361D361E361DBE03D0020E00
:104050001A60F5D71AA01D9ED8901A321AC015F012
:10406000166A176A186A15C018F0176A166A156A70
:1040700015501B1216501C1217501D1218501E12EC
:104080001950D8A414AE01D01E8E1BC011F01CC054
:1040900012F01DC013F01EC014F01200E80E116ED5
:1040A000FF0E126E17ECAFF0000E2F6E300E8CEC80
:1040B000ABF0680E336EE40EE82EFED7332EFCD73D
:1040C00000D0320E50ECB3F0000E2F6E300E8CECA0
:1040D000ABF0150E336EC60EE82EFED7332EFCD78E
:1040E00000D0330E50ECB3F0000E2F6E300E8CEC7F
:1040F000ABF0150E336EC60EE82EFED7332EFCD76E
:1041000000D0340E50ECB3F0000E2F6E250E8CEC68
:10411000ABF0150E336EC60EE82EFED7332EFCD74D
:1041200000D0350E50ECB3F0010E2F6E280E8CEC43
:10413000ABF0150E336EC60EE82EFED7332EFCD72D
:1041400000D0360E50ECB3F0010E2F6E080E8CEC42
:10415000ABF0150E336EC60EE82EFED7332EFCD70D
:1041600000D0370E50ECB3F0010E2F6E010E8CEC28
:10417000ABF0030E346E080E336E770EE82EFED7CA
:10418000332EFCD7342EFAD700F0380E50ECB3F0B3
:10419000010E2F6E060E8CECABF0150E336EC60EB4
:1041A000E82EFED7332EFCD700D0390E50ECB3F0FA
:1041B000010E2F6E0C0E8CECABF0150E336EC60E8E
:1041C000E82EFED7332EFCD700D0410E50ECB3F0D2
:1041D0001200000E226E18AE12D0181E171E161EE8
:1041E000151E141E131E121E116C000E1222132215
:1041F00014221522162217221822010E226E20AE3A
:1042000010D0201E1F1E1E1E1D1E1C1E1B1E1A1E31
:10421000196C000E1A221B221C221D221E221F2294
:10422000202219501A101B101C101D101E101F10D8
:104230002010D8B43CD0010E216E0AD0D890193687
:104240001A361B361C361D361E361F362036212ADE
:1042500020AEF4D71950115C1A5012581B50135845
:104260001C5014581D5015581E5016581F501758E2
:1042700020501858D8A010D01950115E1A50125A58
:104280001B50135A1C50145A1D50155A1E50165AC2
:104290001F50175A2050185AD89020321F321E3201
:1042A0001D321C321B321A321932212ED3D7225022
:1042B000D8B410D0181E171E161E151E141E131E5D
:1042C000121E116C000E1222132214221522162225
:1042D0001722182211C011F012C012F013C013F0EF
:1042E00014C014F015C015F016C016F017C017F062
:1042F00018C018F0120011C018F012C019F013C045
:104300001AF014C01BF01506D8A0160615280FE1E8
:104310001628D8A40CD0000E126E000E116E1200DA
:10432000184A192A1A4A1B2A1506D8A01606600030
:1043300063F0F6FF600067F0F7FF000EF86E1F0EE7
:10434000F76403D00800F55007D06F00DBFFE1FFF2
:104350006F00DFFFE2FFE7500009D8B435D06000FE
:104360006BF0F6FF60006FF0F7FF000EF86E0800CC
:10437000F5500009D8B428D015501610D8B424D060
:1043800060006BF0F6FF60006FF0F7FF000EF86E54
:1043900008006F00D4FF17F0600063F0F6FF6000C4
:1043A00067F0F7FF000EF86E1F0EF76403D00800E9
:1043B000F55007D06F00DBFFE1FF6F00DFFFE2FF8A
:1043C000E7501718D8B4ACD7600063F0F6FF600070
:1043D00067F0F7FF000EF86E1F0EF76403D00800B9
:1043E000F55007D06F00DBFFE1FF6F00DFFFE2FF5A
:1043F000E750176E60006BF0F6FF60006FF0F7FF9C
:10440000000EF86E0800F550175C116E126AD8A005
:1044100012061200400E1CECA8F0030E366E080EB9
:10442000356E770EE82EFED7352EFCD7362EFAD70E
:1044300000F0000E386E000E376E33043410D8A42E
:1044400008D0680E116EF50E126E17ECAFF014EC7A
:10445000B3F0000E3A6E000E396E33043410D8A457
:1044600023D039503A10D8B41FD039C035F0070ED8
:104470003516D8A419D037C035F038C036F0D890EA
:1044800035363636D89035363636D89035363636D7
:10449000680E3524116EF50E3620126E17ECAFF053
:1044A000374A382A14ECB3F0F50E3924F66EF30EC1
:1044B0003A20F76EF86A000EF8220800F55015EC65
:1044C000AAF033043410D8A40FD0F50E3924F66EB8
:1044D000F30E3A20F76EF86A000EF8220800F55045
:1044E000AFECB1F014ECB3F0394A3A2A3A5004E197
:1044F000400E395CD8A0B1D7800E1CECA8F0D00ECD
:10450000356ECA0EE82EFED7352EFCD7120093EC7E
:10451000B3F00009D8A409D02CD08CECB3F0120071
:10452000FCECB3F01200000E120018C11CF019C10F
:104530001DF020EE09F101D80AD00500FA6EDE5018
:10454000FD6EDE50FE6EDE50FF6EFA5012001E6EE3
:104550001F6A1F50000AD8A4E6D71E50010AD8B41B
:10456000E2D7030AD8B4D9D7010AD8B4D9D7070AF1
:10457000DAD7AEECB3F00009D8B435D00101295137
:10458000030B0009D8B40CD0010E1E6E2951030B89
:104590001F6E1E501F5E29511F18FC0B1F18296F1C
:1045A00060008FF4D9FF600093F4DAFFDF50226ED1
:1045B000234B242B2507D8A0260725512611D8A444
:1045C00007D0EEECABF01E6E1E50206E216A04D0B8
:1045D000000E216E030E206E20C023F02250C0EC8E
:1045E000B3F023501200030E1200000E3814000125
:1045F000606F000E3914616F800E3A14626F7F0E87
:104600003B14636F6051611162116311D8A408D02B
:10461000000E386E000E396E000E3A6E000E3B6EC4
:10462000000E3C14606F000E3D14616F800E3E144E
:10463000626F7F0E3F14636F6051611162116311ED
:10464000D8A408D0000E3C6E000E3D6E000E3E6EEB
:10465000000E3F6E3BAE09D0386C391ED8B0392AF7
:104660003A1ED8B03A2A800E3B563FAE09D03C6C79
:104670003D1ED8B03D2A3E1ED8B03E2A800E3F5681
:10468000000E381A000E391A000E3A1A800E3B1A24
:10469000000E3C1A000E3D1A000E3E1A800E3F1A04
:1046A0003C50385C3D5039583E503A583F503B588A
:1046B000D8B002D0D8901200D88012006F00D8FF76
:1046C00009F06F00DCFF0AF06F00E0FF0BF06F00F5
:1046D000D4FF0CF0BE0E0D6EFF0E0E6E3A0167A1F8
:1046E00034D0000E0F6E3901A3A9FDD70F500D2451
:1046F000076E000E0E20086E60001FF0F6FF6000CF
:1047000023F0F7FF000EF86E08006F00D7FFEAFDF8
:104710000F2A060E0F64E7D7BA98000E476E000EF8
:10472000466E000E0101906F000E8F6F46C003F0C1
:1047300047C004F0A5ECB0F08FC103F090C104F0C5
:104740008BECB0F0000E3A01676F57A313D0010154
:10475000AF51D8A40FD04FECACF003C0CBF104C0E4
:10476000CCF105C0CDF106C0CEF1010EAF6F000E49
:104770003A01576F600033F0F5FF60002FF0F8FF4B
:1047800060002BF0F7FF600027F0F6FF110020EE2D
:1047900021F0070EDE6AE806FDE219501A101B1020
:1047A0001C101D101E101F102010D8B446D0010E72
:1047B000296E0AD0D89019361A361B361C361D368B
:1047C0001E361F362036292A20AEF4D7D89021363F
:1047D00022362336243625362636273628361950F3
:1047E000115C1A5012581B5013581C5014581D506D
:1047F00015581E5016581F50175820501858D8A03A
:1048000011D01950115E1A50125A1B50135A1C50D5
:10481000145A1D50155A1E50165A1F50175A205020
:10482000185A2180D89020321F321E321D321C327D
:104830001B321A321932292EC9D721C011F022C0D9
:1048400012F023C013F024C014F025C015F026C0C8
:1048500016F027C017F028C018F0120036C11BF060
:1048600037C11CF038C11DF039C11EF011C01BF05A
:1048700012C01CF013C01DF014C01EF01BC015F0B8
:104880001CC016F01DC017F01EC018F0180E05D081
:10489000D8901832173216321532E82EF9D7155043
:1048A000196E1A6A19501A10D8A419D0D8901B344E
:1048B000156E1C34166E1D34176E1E34186E15508E
:1048C000161017101810D8A405D0000E126E020E84
:1048D000116E1200000E126E030E116E12001928D6
:1048E0001A10D8A41CD01BC015F01CC016F01DC097
:1048F00017F01EC018F0090ED89015361636173668
:104900001836E82EF9D71550161017101810D8A41D
:1049100002D0010E01D0000E116E126A1200000EBC
:10492000126E040E116E1200133414341A6E1A50E3
:10493000D8A409D0000E116E000E126E000E136E78
:10494000000E146E120011C015F012C016F013C044
:1049500017F014C018F0200E05D0D8901832173276
:1049600016321532E82EF9D71550196E138EFF0E38
:104970001116FF0E1216FF0E1316000E1416960EC9
:104980001A5E1AAE0DD01A50800A970FD8A0D2D74F
:10499000D89014321332123211321A3EF9D70DD098
:1049A0001F0E1A6407D0C6D7D890113612361336A8
:1049B00014361A061A50D8A4F7D71950D8B408D00C
:1049C000141E131E121E116C000E1222132214222A
:1049D00011C011F012C012F013C013F014C014F083
:1049E0001200000EBA6E000EBB6E000EBC6EEF0E13
:1049F000C26EC368810EC46E660E3A01606F000E0F
:104A0000506F000E406F000E816F000E516F000E50
:104A1000416F000E616FC49ABC9AC296BA964099D3
:104A2000C298C298BA88C480000E456F000E466FC7
:104A3000000E476F000E656F000E666F000E676F09
:104A4000000E5A6F000E5B6F000E6A6F000E6B6FE8
:104A5000000E426F000E526F180E626F4369536969
:104A60006369446954696469080E846F000E106FAD
:104A7000090E126F0A0E116F0B0E0D6F0C0E086FE0
:104A8000140EE26F210E136F220E146F130E166FA9
:104A9000170EE56F130EE16F1200DC0EF66E630E5B
:104AA000F76E010EF86E00EED0F210EE26F009005F
:104AB0006F00D7FFEEFFE550E150F9E18A0EF66E88
:104AC000660EF76E010EF86E00EED5F110EE15F0E1
:104AD00009006F00D7FFEEFFE550E150F9E1140E39
:104AE000F66E680EF76E010EF86E09006F00D4FFC7
:104AF0004EF009006F00D4FF4FF001EE00F0800E81
:104B0000EE6AE806FDE100EE00F3F00EEE6AE8065C
:104B1000FDE100EE00F2D00EEE6AE806FDE100EEE7
:104B200000F1D50EEE6AE806FDE10001FF6BFE6BB9
:104B300000EE40F00E0EEE6AE806FDE1080ED56EBE
:104B4000000ED66E000ED76E0001BBEF8AF0195032
:104B50001A101B101C101D101E101F102010D8B48E
:104B60003CD0010E216E0AD0D89019361A361B3669
:104B70001C361D361E361F362036212A20AEF4D7AD
:104B80001950115C1A5012581B5013581C501458CD
:104B90001D5015581E5016581F50175820501858A1
:104BA000D8A010D01950115E1A50125A1B50135A27
:104BB0001C50145A1D50155A1E50165A1F50175A81
:104BC0002050185AD89020321F321E321D321C320B
:104BD0001B321A321932212ED3D711C011F012C054
:104BE00012F013C013F014C014F015C015F016C065
:104BF00016F017C017F018C018F012001350141058
:104C0000D8B404D013501410D8A404D011500BEC15
:104C1000B4F0120020EE09F01350D9261450DA2215
:104C2000DE50DE10D8B416D020EE09F01350D9268D
:104C30001450DA2210EE03F01350E1261450E22251
:104C4000DE50E65CE650800A196EDE50800A195884
:104C5000D8B0120020EE03F01350D9261450DA22F7
:104C60006F0078FF15F06F0074FF16F060004FF0D2
:104C7000D9FF600053F0DAFF6F0078FF17F06F0084
:104C800074FF18F015501724D96E16501820DA6EDC
:104C9000600047F0DFFF20EE03F01350D9261450D8
:104CA000DA22DE2A000EDD221200FE6F3F011F9F76
:104CB000CB0E0101836F010E846F60000FF6D9FFE8
:104CC000600013F6DAFF6F004BFCDFFF20EE01F00F
:104CD0008351D9268451DA226F004FFCDFFF20EE8A
:104CE00002F08351D9268451DA226F0053FCDFFF92
:104CF00020EE03F08351D9268451DA22000EDF6EB4
:104D0000D890CB35FA6FCC35FB6FCD35FC6FCE35F7
:104D1000FD6FFE05D8A4120048C0EAF149C0EBF1CE
:104D20007A0EEC6FFE0EED6FFAC1EEF1FBC1EFF102
:104D3000FCC1F0F1FDC1F1F168ECADF048C011F03B
:104D400049C012F061ECAEF0120035503610D8A414
:104D500004D0000E366E010E356E35504E5C4F504D
:104D6000800A386E3650800A3858D8B004D04EC009
:104D700035F04FC036F033043410D8A404D0355089
:104D80007F0F1CECA8F0020E33183410D8A404D006
:104D90003550BF0F1CECA8F0030E33183410D8A404
:104DA00004D03550930F1CECA8F0040E33183410C7
:104DB000D8A404D03550D30F1CECA8F0150E386ED3
:104DC000C60EE82EFED7382EFCD700D0375015EC93
:104DD000AAF0150E386EC60EE82EFED7382EFCD778
:104DE00000D0120040504110D8A405D040C020F09F
:104DF00041C021F006D0FF0E4024206EFF0E41205E
:104E0000216E44A009D01CC011F0126A1AC013F020
:104E10001BC014F0FEECA5F021AE04D0000E216EF4
:104E2000000E206E000E1F6E000E1E6E0CD0000EC7
:104E3000126E200E116E1AC013F01BC014F0FEEC9F
:104E4000A5F01E4A1F2A20501E5C1F50800A1D6EAE
:104E50002150800A1D58D8A0EAD744B009D01CC000
:104E600011F0126A1AC013F01BC014F0FEECA5F08A
:104E7000010E1E241A6E000E1F201B6E1200116EF2
:104E8000010E126E010129B745D011C022F12995FA
:104E90002987FC0E29170F0E276F010E216FF40EC4
:104EA000206F2989040E006F680E016F010E026FDA
:104EB000000E126F000E136F040E036F680E046F66
:104EC000010E056F000E146F000E156F040E066FB5
:104ED000680E076F010E086F000E166F000E176F39
:104EE000040E096F680E0A6F010E0B6F000E186F2B
:104EF000000E196F000E0C6F680E0D6F010E0E6F15
:104F0000000E1A6F000E1B6FE4ECB3F036ECB2F03B
:104F1000000E126E1250120044A00AD023C01AF0E4
:104F200024C01BF021C01CF022C01DF007ECB0F023
:104F300026BE05D025C02AF026C02BF004D0000ED6
:104F40002B6E000E2A6E000E296E000E286E0CD0FD
:104F5000000E126E200E116E21C013F022C014F04C
:104F6000FEECA5F0284A292A2A50285C2950800AFC
:104F7000276E2B50800A2758D8A0EAD744B00AD011
:104F800023C01AF024C01BF021C01CF022C01DF069
:104F900007ECB0F023C011F024C012F03BECAEF0EF
:104FA0002A501124216E2B501220226E1200000E66
:104FB0001114196E000E12141A6E800E13141B6E4B
:104FC0007F0E14141C6E19501A101B101C10D8A43C
:104FD00008D0000E116E000E126E000E136E000E41
:104FE000146E000E1514196E000E16141A6E800E33
:104FF00017141B6E7F0E18141C6E19501A101B10FC
:105000001C10D8A408D0000E156E000E166E000EEF
:10501000176E000E186E155011180AE1165012186E
:1050200007E11750131804E118501418D8B402D02F
:10503000D8901200D8801200316E270E0001FF6F49
:105040003150F00B0C09326E32C02BF0FF51DAEC0C
:10505000B1F03150F00B0809326E32C02BF0000174
:10506000FF51DAECB1F031C02FF00F0E2F162F38B0
:10507000F00B0C09326E32C02BF00001FF51DAEC5C
:10508000B1F031C02FF00F0E2F162F38F00B08099A
:10509000326E32C02BF00001FF51DAECB1F0310476
:1050A000D8A41200020E306EA00E2F6E920EE82EC3
:1050B000FED72F2EFCD7302EFAD700D01200000ECC
:1050C000166E14AE06D0136C141ED8B0142A010E3E
:1050D000166E12AE06D0116C121ED8B0122A010E36
:1050E000161A000E186E000E176E13501410D8B456
:1050F0001CD0010E156E04D0D89013361436152A24
:1051000014AEFAD7D890173618361350115C1450D5
:105110001258D8A005D01350115E1450125A17809F
:10512000D89014321332152EEDD71650D8B404D0BF
:10513000176C181ED8B0182A17C011F018C012F03A
:105140001200000E196E000E1A6E000E1B6E000E7D
:105150001C6E1550161017101810D8B42AD0010E56
:105160001D6E06D0D89015361636173618361D2AFD
:1051700018AEF8D7D89019361A361B361C3615508B
:10518000115C165012581750135818501458D8A0C4
:1051900009D01550115E1650125A1750135A185054
:1051A000145A1980D89018321732163215321D2E23
:1051B000E1D719C011F01AC012F01BC013F01CC0C7
:1051C00014F01200166E115012101310D8B420D023
:1051D0001650030D000EF324D96E010EF420DA6E82
:1051E000600047F0DEFF60004BF0DEFF60004FF034
:1051F000DEFF1650020D120EF324D96E010EF420BC
:10520000DA6E600053F0DEFF600057F0DDFF120041
:105210001650030D000EF324D96E010EF420DA6E41
:10522000040EDE6E680EDE6E010EDE6E1650020D8E
:10523000120EF324D96E010EF420DA6E000EDE6E2B
:10524000000EDD6E12009AECB3F00009D8A402D073
:10525000040E120001012951030B0009D8B40CD02F
:10526000010E206E2951030B216E2050215E295121
:105270002118FC0B2118296F2507D8A026072551D6
:105280002611D8B40DD0F1ECB3F060008FF4D9FF43
:10529000600093F4DAFFDF6E0101234B242BD8D793
:1052A0009EECA9F0226EF1ECB3F060008FF4D9FF10
:1052B000600093F4DAFFDF6E0101234B242B2250B0
:1052C0001200376E3350D8A402D0010E336E335023
:1052D000346E356A34504E5C4F50800A366E35500D
:1052E000800A3658D8B002D04E04336E3704D8A4A2
:1052F00004D033507F0F1CECA8F0020E3718D8A44E
:1053000004D03350BF0F1CECA8F0030E3718D8A4FC
:1053100004D03350930F1CECA8F0040E3718D8A417
:1053200004D03350D30F1CECA8F0150E346EC60E0B
:10533000E82EFED7342EFCD700D01200298916D0D3
:10534000F4ECB3F0080E1200F4ECB3F0070E120008
:1053500001012529C5ECB3F0040E1200070E01016E
:105360002719D8A4F7ECB3F00F0E120012C11CF0ED
:1053700013C11DF001D80AD00500FA6E0051FD6E70
:105380000151FE6E0251FF6EFA5012001E6E1F6A2E
:105390001F50000AD8A4E2D71E50010AD8B4DED7A5
:1053A000030AD8B4D1D7010AD8B4CAD7070AD8B4E7
:1053B000CFD7D4D73901A3A7110093A711006F004D
:1053C000A0F7C0F10D0E0101C019D8B406D04B50A2
:1053D00004E17F0E4A5CD8A018D0010EBC6F700E9D
:1053E0004A24D96E030E4B20DA6E000EDF6E4AC0DF
:1053F00097F14BC098F1000E4B6E000E4A6E3901CA
:1054000093976F00A0F7C0F11100700E4A24D96E77
:10541000030E4B20DA6E600003F7DFFF4A4A4B2A87
:105420004AC097F14BC098F11100306E270E000171
:10543000FF6F3050F00B0D090101A96FA9C12BF0CE
:105440000001FF51DAECB1F03050F00B0909010115
:10545000A96FA9C12BF00001FF51DAECB1F030C007
:105460002FF00F0E2F162F38F00B0D090101A96F29
:10547000A9C12BF00001FF51DAECB1F030C02FF0E0
:105480000F0E2F162F38F00B09090101A96FA9C1C2
:105490002BF00001FF51DAECB1F01200000E166E95
:1054A00012AE06D0116C121ED8B0122A010E166E62
:1054B00014AE04D0136C141ED8B0142A1350141058
:1054C000D8B418D0010E156E04D0D8901336143607
:1054D000152A14AEFAD71350115C14501258D8A0E4
:1054E00004D01350115E1450125AD8901432133253
:1054F000152EF1D71650D8B404D0116C121ED8B0A6
:10550000122A11C011F012C012F01200000E366EF5
:10551000000E356E14D035503124336E36503220A3
:10552000346E6000CFF0F6FF6000D3F0F7FF000E9E
:10553000F86E0800F55015ECAAF0354A362A3550B9
:105540003124336E36503220346E6000CFF0F6FFD7
:105550006000D3F0F7FF000EF86E0800F550000968
:10556000D8B412004E50355C3650800A336E4F501E
:10557000800A3358D8B01200CED72B6E27C02EF039
:1055800028C02FF029C02CF02AC02DF02B503FEC62
:10559000A7F00009D8B4FAD7D60E176E5B0E186EB6
:1055A000010E196E2C0E1A6E1B6AD2ECB2F0260E8A
:1055B000116E126A000E146E010E136E07ECB3F03A
:1055C000000E176E000E186E000E196E000E1A6E89
:1055D000000E1B6EC4ECB2F0D4ECB3F058ECB2F099
:1055E000E806D8A41200FAD7155016101710181094
:1055F000D8B424D0010E196E06D0D89015361636C0
:1056000017361836192A18AEF8D71550115C1650EF
:1056100012581750135818501458D8A008D01550C5
:10562000115E1650125A1750135A1850145AD89027
:105630001832173216321532192EE7D711C011F071
:1056400012C012F013C013F014C014F01200600066
:105650004FF0F6FF600053F0F7FF000EF86E080001
:105660006F00D4FFAAF119D060004FF0F6FF600080
:1056700053F0F7FF000EF86E08006F00D4FFAAF198
:10568000600047F0D9FF60004BF0DAFF6000ABF636
:10569000DFFF114A122A134A142A0101AA51D8A481
:1056A000E3D7600047F0D9FF60004BF0DAFF000E4F
:1056B000DF6E1200276E000E286E27503FECA7F019
:1056C0000009D8B4FAD7A00E176E620E186E010E3C
:1056D000196E280E1A6E1B6AD2ECB2F0260E116EED
:1056E000126A000E146E010E136E07ECB3F0000E7A
:1056F000176E000E186E000E196E000E1A6E000E58
:105700001B6EC4ECB2F0D4ECB3F058ECB2F0E80687
:10571000D8B4FBD728501200316E3150F00B0C0971
:10572000326E32C02BF0270EDAECB1F03150F00BB4
:105730000809326E32C02BF0270EDAECB1F02F04DC
:10574000D8A4120031C030F00F0E30163038F00BF4
:105750000C09326E32C02BF0270EDAECB1F031C0FA
:1057600030F00F0E30163038F00B0809326E32C0B0
:105770002BF0270EDAECB1F01200F6C0FAF0F7C009
:10578000FBF0000E0101726F000E716F15D0F4C0B6
:10579000C3F0F5C0C4F0FA0E0001C56FF8C0C6F042
:1057A000F9C0C7F000EC80F00001C351010171277E
:1057B0000001C451010172236000EBF3F6FF6000A9
:1057C000EFF3F7FF000EF86E0800F5500009D8A4BB
:1057D000DED771C1F4F072C1F5F0120029890ED044
:1057E000F4ECB3F0070E120001012529C5ECB3F06B
:1057F000030E1200F7ECB3F00A0E120012C11CF0F7
:1058000013C11DF001D80AD00500FA6E0051FD6EDB
:105810000151FE6E0251FF6EFA5012001E6E1F6A99
:105820001F50000AD8A4E6D71E50010AD8B4E2D708
:10583000030AD8B4D5D7060AD8B4D6D7DBD717C051
:105840001BF018C01CF015C01DF016C01EF01B5038
:10585000196E1C501A6E1B4A1C2A600067F0F6FF76
:1058600060006BF0F7FF000EF86E600077F0D9FF74
:1058700060007BF0DAFF1D4A1E2A1F0EF76403D07A
:105880000800F55007D06F00DBFFE1FF6F00DFFF7E
:10589000E2FFE750DF6EDF50D8B41200D8D7CF0E4A
:1058A000836F010E846F60000FF6D9FF600013F65E
:1058B000DAFF6F004BFCDFFF20EE01F08351D926A9
:1058C0008451DA226F004FFCDFFF20EE02F083519B
:1058D000D9268451DA226F0053FCDFFF20EE03F05B
:1058E0008351D9268451DA22000EDF6ECFC103F036
:1058F000D0C104F0D1C105F0D2C106F012003901C7
:10590000A3B76F00A0F7C0F1000E126E000E116E6B
:10591000700E1124D96E030E1220DA6E000EDF6EA7
:10592000114A122A125004E17F0E115CD8A0F0D760
:105930003D01F289000EF96F000EFA6F000E0301AF
:10594000706F000E0101986F000E976F000EC06F10
:10595000000EBC6F3901938D93871200286E28507A
:105960003FECA7F00009D8B4FAD7400E176E620ECC
:10597000186E010E196E270E1A6E1B6AD2ECB2F069
:10598000260E116E126A000E146E010E136E07ECD5
:10599000B3F0000E176E000E186E000E196E000E9A
:1059A0001A6E000E1B6EC4ECB2F0D4ECB3F058ECDF
:1059B000B2F0E806D8A41200FAD7E4ECB3F0020E75
:1059C0000101286F09D08CECB3F01200FCECB3F0AD
:1059D00012007DECB3F0120014C11CF015C11DF0D3
:1059E00020EE03F101D80AD00500FA6EDE50FD6EFC
:1059F000DE50FE6EDE50FF6EFA5012001E6E1F6A01
:105A00001F50000AD8A4E5D71E50020AD8B4DBD72D
:105A1000010AD8B4DBD7DDD780ECB1F00101295100
:105A2000030B0009D8B408D093ECB3F00009D8B444
:105A300003D0100E0101276F01012751030D350E10
:105A4000F324F66EF40EF420F76EF86A000EF822D6
:105A500001D80DD00500FA6E0900F550FD6E090061
:105A6000F550FE6E0900F550FF6EFA50120001016C
:105A7000276F1200000E3E01DE6F000EDF6F000E7A
:105A8000E06F000EE16F000EE46F000EE56F000E98
:105A9000EA6F000EEC6F000EF16F000EF36F000E58
:105AA000F46F000EF56F000EF66F000EF76F000E2C
:105AB000F96F000EFA6F000EFB6F000EFC6F000E08
:105AC000FD6F000EFE6F030EFF6F840EF86F120065
:105AD000EE0E0301FB6F010EFC6FEAC1F0F3EBC1A8
:105AE000F1F3000EF46F000EF36F000EFA6F000E6C
:105AF000F96FF00E0001F46F030EF56FECC1F6F0D4
:105B0000EDC1F7F0FB0EF86F030EF96FBDECABF0D3
:105B10000301F3510101EA25D96E0301F45101019A
:105B2000EB21DA6E000EDF6E1200010E266EFF0E04
:105B3000276E220EAEECACF0050E266EFF0E276E21
:105B4000220EAEECACF0070E266EFF0E276E220E74
:105B5000AEECACF00D0E266EFF0E276E220EAEECF4
:105B6000ACF0090E266E000E276E220EAEECACF0E5
:105B70000B0E266E440E276E220EAEECACF0120019
:105B8000FC0E2917020E286F299505D0FAECB3F008
:105B900012000F0E120016C11CF017C11DF020EEEE
:105BA00006F101D80AD00500FA6EDE50FD6EDE5017
:105BB000FE6EDE50FF6EFA5012001E6E1F6A1F50FE
:105BC000000AD8A4E6D71E50020AD8B4DFD7010ACB
:105BD000D8B4DCD7DED720EE02F01C50D9261D50F9
:105BE000DA226F0078FF11F06F0074FF12F060008E
:105BF00073F0D9FF600077F0DAFF6F0078FF13F0E1
:105C00006F0074FF14F007ECB3F0000E176E000E77
:105C1000186E000E196E000E1A6E000E1B6ED2EC7E
:065C2000B2F0020E1200BA
:105C28006F00E8FF01F06F00ECFF02F03901A39F5D
:105C38006000A3F6B7FF60009FF6B6FF01016E5142
:105C48006F117011D8B40CD001D80AD00500FA6EC3
:105C58006E51FD6E6F51FE6E7051FF6EFA5012005C
:105C680060000BF0FBFF600007F0FAFF110011C0A5
:105C780013F012C014F002D0114A122A600047F043
:105C8800F6FF60004BF0F7FF000EF86E1F0EF7648A
:105C980003D00800F55007D06F00DBFFE1FF6F006D
:105CA800DFFFE2FFE7500009D8A4E6D71350115CE4
:105CB800116E14501258126E1200000E146E000E5F
:105CC800136E16D03901A3A9FDD713501124D96E2C
:105CD80014501220DA6EDF503D01EA6F134A142A7D
:105CE80014BE06D014500EE1810E135CD8B0120019
:105CF80013501124D96E14501220DA6EDF50D8B424
:105D08001200E0D712002A6E2A503FECA7F00009D3
:105D1800D8B4FAD726C011F027C012F028C013F063
:105D280029C014F007ECB3F0000E176E000E186EC1
:105D3800000E196E000E1A6E000E1B6EC4ECB2F047
:105D4800D4ECB3F058ECB2F0E806D8A41200FAD7B5
:105D5800000E3D01EC6F000EED6F000EEE6F000EB1
:105D6800EF6F000EF06F000EF16FB00EF26F800E45
:105D7800F36F000EF46F8A0EF56F000EF66F000ECB
:105D8800F76F000EF86F000EF96F000EFA6FF28BC6
:105D9800F289390193971200000E356E000E346EA9
:105DA8000BD034503124D96E35503220DA6EDF50A2
:105DB80015ECAAF0344A352A34503124D96E3550BE
:105DC8003220DA6EDF50D8B412004E50345C3550B1
:105DD800800A336E4F50800A3358D8B01200E1D78A
:105DE800000E3C1A000E3D1A000E3E1A800E3F1A95
:105DF80038C011F039C012F03AC013F03BC014F0AB
:105E08003CC015F03DC016F03EC017F03FC018F07A
:105E180030EC95F011C038F012C039F013C03AF0E8
:105E280014C03BF0120011D03901A3A9FDD76000BE
:105E380047F0F6FF60004BF0F7FF000EF86E080021
:105E48006F00D7FFEAFD114A122A600047F0F6FFFB
:105E580060004BF0F7FF000EF86E0800F5500009DF
:105E6800D8B41200E1D7D29ED28A550ED46EAA0EAB
:105E7800D46ED490000ED76E000ED66E080ED56E76
:105E8800550ED46EAA0ED46ED48039018387808FC4
:105E98008485899181918491839F8495D28CD28EB7
:105EA800D29E120039019991050E966E800E956E5C
:105EB800010E976E94508F0B5009946E9450F00B0E
:105EC8000609946EDF0E936E000E0101B86FB59B44
:105ED800000E886F000E876F3901A9919981948E01
:105EE8001200010E176E200E11181210D8B414D01B
:105EF800F70E136EFF0E146E11C015F012C016F0D7
:105F08001350152614501622165004E1050E155C80
:105F1800D8A002D0000E176E17C011F0126A120036
:105F2800246E010E256E010129B516D02985000EB3
:105F3800256E2551C5ECB3F02450D8B406D0040E14
:105F48000101276F47ECB2F005D0030E0101276F5E
:105F58005AECB3F064ECB3F025501200BF0E196E82
:105F6800FF0E1A6E17C01BF018C01CF019501B2624
:105F78001A501C221C500AE11A0E1B5CD8B006D01D
:105F8800200E1710176E1850186E120017C017F051
:105F980018C018F012003F011E991E971E951E93F7
:105FA8001E911E8F1E9B1F9F1F9D2185219321914E
:105FB8003901A19D919DA19B919B3F011D691C6980
:105FC8001B691F971F951F931F911E8F12009F0E0D
:105FD800196EFF0E1A6E17C01BF018C01CF019506E
:105FE8001B261A501C221C5009E11A0E1B5CD8B043
:105FF80005D05F0E1714176E186A120017C017F035
:1060080018C018F01200000E206E000E1F6E0BD084
:106018001EC011F0126A1CC013F01DC014F0FEEC73
:10602800A5F01F4A202A1F501A24D96E20501B2081
:10603800DA6EDF501E6E1E50D8B41200E9D7000E7B
:10604800166E000E156E0ED0520E146E2B0E136EB9
:10605800000EE82EFED7132EFCD7142EFAD700D048
:10606800154A162A1150155C12501658D8B012004D
:10607800EBD79F0E136EFF0E146E200E1110156EC7
:10608800000E1210166E13501526145016221650B4
:1060980006E11A0E155CD8B002D0010E01D0000E30
:1060A800116E126A1200FF0E1116030E12167AA84C
:1060B8000DD0060ED89011361236E82EFBD76000A8
:1060C8004BF079FF600047F078FF120060004BF05A
:1060D80079FF600047F078FF1200FF0E1116030EDB
:1060E80012167EA80DD0060ED89011361236E82E5C
:1060F800FBD760004BF07DFF600047F07CFF12008B
:1061080060004BF07DFF600047F07CFF1200FF0E3F
:106118000316030E04167AA80DD0060ED89003367F
:106128000436E82EFBD7600013F079FF60000FF00B
:1061380078FF1200600013F079FF60000FF078FF1D
:106148001200FF0E0316030E04167EA80DD0060ECD
:10615800D89003360436E82EFBD7600013F07DFF95
:1061680060000FF07CFF1200600013F07DFF6000FC
:106178000FF07CFF120024BE05D0245010E1230448
:10618800D8B00DD023C025F024C026F0251E261E29
:10619800254A262A25C023F026C024F0120023C051
:1061A80023F024C024F012009F0E136EFF0E146E0D
:1061B80011C015F012C016F01350152614501622EF
:1061C800165006E11A0E155CD8B002D0010E01D0A7
:1061D800000E116E126A1200BF0E136EFF0E146EBF
:1061E80011C015F012C016F01350152614501622BF
:1061F800165006E11A0E155CD8B002D0010E01D077
:10620800000E116E126A1200D00E136EFF0E146E7D
:1062180011C015F012C016F013501526145016228E
:10622800165006E10A0E155CD8B002D0010E01D056
:10623800000E116E126A12001CC011F01DC012F07F
:10624800000E146E010E136E07ECB3F0000E176EFD
:10625800000E186E000E196E000E1A6E000E1B6EE0
:10626800D2ECB2F0040E12001CC011F01DC012F0E6
:10627800000E146E020E136E07ECB3F0000E176ECC
:10628800000E186E000E196E000E1A6E000E1B6EB0
:10629800D2ECB2F0020E12001CC011F01DC012F0B8
:1062A800000E146E010E136E07ECB3F0000E176E9D
:1062B800000E186E000E196E000E1A6E000E1B6E80
:1062C800D2ECB2F0020E12001CC011F01DC012F088
:1062D800000E146E020E136E07ECB3F0000E176E6C
:1062E800000E186E000E196E000E1A6E000E1B6E50
:1062F800D2ECB2F0040E1200A1ECB3F00009D8B44D
:1063080003D008ECB4F01200B4ECB3F00009D8B430
:1063180003D004ECB4F01200BAECB3F00009D8B41E
:10632800120006ECB4F012001150121013101410E1
:10633800D8B408D0000E111A000E121A000E131A43
:10634800800E141A11C011F012C012F013C013F00D
:1063580014C014F01200126E800E0ED012501314D6
:106368000009D8B404D02A0E50ECB3F003D0200EA4
:1063780050ECB3F0D8901330136E1350D8B4120009
:10638800EDD7115013026F00CCFF15F06F00D0FF4E
:1063980016F011501402F350162612501302F3503F
:1063A800162615C011F016C012F012002C6E2BC064
:1063B8002DF0000E2E6E2D0E266E276A000E296E09
:1063C800010E286E2C5087ECAEF01A0EE82EFED780
:1063D80000D012009AF65FF6FCF623F746F727F589
:1063E80023F6A8F576F4E6F57AF7D2F600FF000072
:1063F80000FF00FF00FF2C2C00FF1FC011F020C081
:1064080012F03BECAEF011501F24156E12502020F4
:10641800166E21C017F022C018F01FECACF0120065
:10642800000E0101CB6F000ECC6F000ECD6F000E79
:10643800CE6FCB0E836F010E846F3F01208B1F8FB1
:106448001200030E3D017B6F040E736F800E746F94
:10645800000E756F000E6C6F7599200E6E6F799532
:10646800739F120073BF1200000E796F000E7A6FCF
:10647800000E766F6C69510E3A016A6F510E6B6FA0
:106488003D01738F120001012951FC0B0209296F8C
:1064980025052611D8B49EECA9F0D8800101223533
:1064A800C0ECB3F0040E1200010E116E010129B503
:1064B8000AD029972269E4ECB3F099ECB2F0CFEC5A
:1064C800B3F028C111F0115012003D017995600018
:1064D80047F06EFD000E6C6F738B79A5FED774BB09
:0A64E80002D0010E1200000E120097
:1064F4006F0060FF10F00101874B882B010EB86F0D
:10650400DF0E936E3901A991600043F0D8FF1100AA
:10651400E8ECB3F0FEECB3F00009D8B406D0000EFA
:10652400C5ECB3F0000EC0ECB3F0000E120039015C
:1065340093939395929F93913D017A917A957A9F43
:106544007A9D7A937693769576911200010EA26ED7
:10655400000EA16E000EA36E9F68000E9E6E3901A0
:10656400A791C00EA06E1200010EAE6E000EAD6EAD
:10657400000EAF6EAB68000EAA6E3901A495C00E72
:10658400AC6E120017C011F018C012F019C013F04D
:106594001AC014F01BC015F0020EE2ECA8F01200B1
:1065A40017C011F018C012F019C013F01AC014F07B
:1065B4001BC015F0000EE2ECA8F012003B6E38C0D0
:1065C40033F03B5061ECA9F039C031F03AC032F0FD
:1065D40086ECAAF012003B6E38C033F03B5061ECFD
:1065E400A9F039C031F03AC032F0D0ECAEF012006C
:1065F4003901A3B11200A2BF12003D0179B5120006
:1066040079BF120076B91200F3D7010129A912004B
:1066140011C023F112C024F113C025F114C026F1D6
:10662400299912003901A3A9FDD70D0E3D01EA6F86
:106634003901A3A9FDD70A0E3D01EA6F12008C0EA1
:106644007E6E000E7D6E000E7C6E3F015E51FC0B73
:0666540001095E6F120057
:10665C003901A4A51100A495010E0101AE6F7D4B6B
:10666C007E2BF90EAB6E11008C0E7A6E000E796ECD
:10667C00000E786E5E51F30B08095E6F1200286EE7
:10668C00756C6C2900010002000400080010000069
:03669C008020203B
:1066A000116E01D000F03901A3A9FCD7600047F0BA
:1066B000EAFD12002951FC0B0209296F2251222503
:1066C000C0ECB3F0030E120004D0FAECB2F00CEC04
:1066D000ADF0010129A51200F8D7130E266E220E87
:1066E0005AECABF0296E29501200CAECB3F001014C
:1066F0002995020E286F0F0E1200CAECB3F00101AB
:106700002995000E286F0F0E1200EBECB3F0E8ECA9
:10671000B3F0A8ECB3F0120001012551C5ECB3F0C1
:1067200047ECB2F012003D0174AB02D0010E120032
:10673000000E12003D0178A102D0010E1200000EE1
:1067400012003D0179AF02D0010E1200000E1200BE
:1067500001012995000E286F0F0E120078AB02D0B0
:10676000010E1200000E120079A502D0010E1200D7
:10677000000E120076A902D0010E1200000E1200C7
:10678000116E600047F06BFD1200116E600047F063
:106790006CFD12003D01739F7885738F1200739F0B
:1067A000000E796F78851200000E94ECAFF01200A5
:1067B000EBECB3F0090E1200EEECB3F0040E120095
:1067C000EEECB3F0030E1200000E3D01796F1200E3
:1067D0003D01739B12003D01748D12003D01749DBB
:1067E00012003D016A5112003D01738D12003D01FE
:1067F000739D1200010E1200020E12006C51120065
:10680000050E1200010E1200799512007699120001
:0C681000799F1200140012001100120009
:020000040020DA
:10000000FFFFFFFFFFFFFFFFFFFFFFFFFFFFFFFF00
:020000040030CA
:0A0000008CFFFFFF8DFFFFFFFFFFE5
:00000001FF
